:020000041100E9
:103000000023F7B52E4D2F4C280063616374022610
:1030100001F07AF94021FE22217428002A4B009603
:1030200001F0C4F900283AD1217CFF222800274B67
:10303000009601F0BBF9002831D1254BA2899A42B4
:103040002AD1E389234A934211D1234B6361234B55
:103050002268002A07D1002B05D019002200C1C91F
:10306000C1C21B7B6374280001F08CF9F7BD1C4AB8
:10307000934201D00023EBE71A4B1B4A1B68934293
:1030800006D9C02304222800217C9B0001F004FA09
:10309000164B6361164BDBE700232374EAE7CC236E
:1030A0003821AC2228009B01217401F0F5F9002899
:1030B000F2D1104B6361104BE381104BC8E7C0465F
:1030C000D441FF1F9461FF1FA061FF1FA261FF1F7A
:1030D0005959000083050000394100117CB90011E5
:1030E00082150000B861FF1F87130000ED41001139
:1030F0008CB9001185410011AAAAFFFF6CB900111B
:10310000F7B5164B0192C318021D002000938823C7
:103110005B05D3181B685C1C1AD09CB2402C18D8D5
:103120008D781E0CAC466746CD782D023D43AE42ED
:1031300006D1019800280ED110000C70240A4C70A2
:1031400003249BB20733A343D218009B9A42DED3D9
:10315000FEBD4432F9E71000FAE7C046FC0F00005C
:10316000802213B503000324019189B25201073173
:103170009B18A14304305A1A88235B05C3181B68A7
:10318000591C03D190429241104016BD99B240297A
:1031900007D80B000733A343C0189042ECD300209C
:1031A000F3E74430F9E7134B134A1B68126810B574
:1031B000FA24934201D81A00F824104BE4021B6849
:1031C0009A4210D813000E4A12689A420ED3013365
:1031D00007D1F823DB029C4203D10A49054808F0D5
:1031E0003FF9200010BDFC24E402ECE7FE24E402D9
:1031F000F7E7C04600C0071100D0071100E0071133
:1032000000F00711FFFFFF7FF0B59BB015000490A1
:103210000391402A00D9A0E006AB59801A80FFF73D
:10322000C2FF0400042816D9002206A9FFF768FF90
:10323000052810D906AB1B88AB420CD1002D07D056
:10324000514B2A000499C01808F012F8002802D146
:1032500001201BB0F0BD06AB1D8020000699FFF7D2
:103260007FFF041E7BD1069B0793FFF79CFF802303
:103270005B01C618802307001B039E4201D3F8267A
:10328000F60288235B05F31801931B68013302D013
:10329000019808F01DF83D49019808F0E1F83B1D40
:1032A0000293331D05938822029B52059B181B68CD
:1032B00008935A1C3CD044219AB20091402A04D869
:1032C0000320D11D814389B2009103991B0C8B42CD
:1032D00024D0402A22D80122300008A9FFF710FF8D
:1032E000021E1BD1380008A9FFF70AFF04000428BA
:1032F00031D9009A059B9B1880225201B218934243
:1033000040D288235B05C118009A09A808F060F82C
:103310001D4B009A09A9F01808F022F8009A029BA8
:103320009446634402931A4B029AFB189A42BAD30A
:1033300088235B05FC1821680198013908F090F892
:10334000200007F0C5FF039A07AB5A8030000799A9
:10335000FFF706FF0400002C03D1002079E70428C2
:10336000FBD988235B05E018069908F079F8032358
:10337000EA1C9A4300D16BE7034B0499E01807F06D
:10338000EFFF65E70424ECE704000011FFFFFF7F77
:10339000F80F0000F7B505001400402A21D80027D7
:1033A00001AE71803780FFF7FEFE042816D93A007F
:1033B0003100FFF7A5FE042810D93688BC420BD097
:1033C000BD4209D0221CB44200D9321C064B92B235
:1033D000C118280007F0FCFF30B2FEBDC04300B2A8
:1033E000FBE703204042F8E70400001137B5042250
:1033F00004000D0001A81649FFF7CCFF02000428C5
:103400000BD1019BA34208D3AB4204D0104901A8C1
:103410000195FFF7F9FE01203EBD0E4C2368200008
:10342000019307F055FF019920000139019108F03F
:1034300017F880235B01E418074B9C42EED104226D
:10344000034901A80195FFF7DFFE0020E4E7C0462D
:103450005555000000C007110000081130B589B0B3
:1034600008F016F810226946254808F0C9F9254BDE
:10347000009A9A420ED1019B029A0F2B33D8002159
:1034800001240698013B08D2002900D00292029B39
:10349000013331D10023029325E0551CF2D1020003
:1034A0002100EFE710341022200004A908F0A8F949
:1034B000029B013301D1069B0293882304995B058B
:1034C000C918059B06981A03120B049105928142B4
:1034D00003D02B4201D107F07BFF019B013B0193FD
:1034E000019B002BDED1029B002B03D00493049898
:1034F0004168084709B030BDE025014C2D03EFE7D6
:1035000000000111504859368022F8B5964C974B6F
:10351000D200002120001C6008F052F92300944AD8
:1035200088331A60934B1A786A23002A00D011332B
:10353000E3620A232365904B37221B780820A3639C
:103540008E4B2118E361102323628D4B3B25636171
:10355000C823DB00A36123008C331A602823013ABF
:10356000E26320646364CA67043A211DCA672100CC
:10357000BC310D602100C03108602100C4310B60F6
:1035800021000635CC310D602100083DC8310D60A9
:103590002100D0310A602200D43210602200D832DB
:1035A000136022000227E032210017604222DC3142
:1035B0000A6021001B3DE4310D602100E831086004
:1035C0002100EC310B6023000521F4331960230046
:1035D000F0331A602300183290331A6023009433BA
:1035E000186023001E3A98331A60AF23DB00236073
:1035F000644BFA262363644B644DE360644BF03103
:10360000A3642300FF31FC33B600A16021611E607A
:10361000A5627325E5656D3D6565A56596255D4AE1
:10362000AD00E264666258606766A56600270925FA
:10363000A767E566584F594D606720002567E26728
:103640003A6015279C30676007001A203860200018
:10365000A0300700212038602000A83007004C4827
:1036600038602000F830066026006427A4363760F2
:1036700026005F3FAC3637602600033FB036376028
:103680002600C637B436376026000027B8363760C4
:1036900038269E60424E96205E64424E5A66DE6137
:1036A000414E9A645E62F53EFF3E9E621E269A6718
:1036B000354A8000DE661F675F67DD651D6618623C
:1036C000DA67BE23394A5B00E250394BD8382350C1
:1036D00004302250C4225200A350C623E4205B00D1
:1036E000E1500433334AE1503349344BD16034491B
:1036F000800019503349E938FF38195032490430F5
:10370000195032493248D16132491163324951630B
:103710001900F4310860CE20304940001160304972
:10372000195019002F48F83108602F49D1658221BE
:103730002E4A89005A501A002D490832D1671A00C2
:103740002C49B432116088212B4A89005A501A0042
:103750002A49883211602A4ADA6407F0A1FE012062
:1037600007F0CEFFF8BDC0460004FF1F3064FF1F06
:10377000006FFF1F0444FF1F4A0AFF1F3A070000A3
:1037800080C3C9019A020000DC0500006A1800002D
:1037900050C3000088130000F009FF1F204E0000F6
:1037A0006509FF1F68100000C409000040420F00B7
:1037B00010270000FC00FF1F751CFF1F0000FF1FEB
:1037C000C92CFF1F5130FF1FE92EFF1F3520FF1F9F
:1037D0002527FF1F5120FF1FFD21FF1FC11FFF1FB6
:1037E0004929FF1F312AFF1F8D19FF1F5528FF1F71
:1037F0007925FF1F8525FF1FC11EFF1F791FFF1F92
:10380000391EFF1F0223F0B50124644D644E2B7056
:10381000644B91B01C70644F0393336800210820FF
:10382000BB7006F00FFC082006F006FB0023984250
:1038300005D0BA78552A02D0332A00D0A1E03360EF
:10384000042006F079FD07F0EBFEFFF75DFE07F0C0
:103850007FFF1F2201240021544B10AE1A70544BDD
:103860001C70544B1970544B19689143163A0A4313
:103870001A60602219689143403A0A431A6007F0BF
:103880009FFD07F0E5FD4D4B9847C120FF214C4BB4
:1038900080001A588A431A50C522920098588843CB
:1038A000BF39014399509858464908408021C901C1
:1038B0000143802099509958C0050902090A014323
:1038C000995080214048490107F06AFE03232200F5
:1038D0003E49019400933E4807F032FE2C223D49B8
:1038E00005A807F075FD05AC61782078023406F074
:1038F000C3FAA642F8D1384C0121002006F0D0FBD3
:103900000920012106F0CCFB2268344B03201A4029
:10391000A023DB0213432360802322689B0413430C
:10392000236022682E4B1A4080239B03134323609D
:103930002C4A2D4B934200D8012007F0F9FD07F0E7
:1039400097FF80232268DB0413432360287807F065
:1039500007FE039B1878C0B207F082FF07F0C8FD8E
:103960002249042007F0A4FE06F0B2FC00F040F863
:1039700000F0BEFD00F066FE00F00CFA002011B071
:10398000F0BD00932100194A042007F019FE80239E
:10399000DB059C62FFF762FD52E7C0464A0AFF1F43
:1039A00034F000400444FF1FC461FF1F480AFF1F9A
:1039B000490AFF1F680AFF1FBCF00040E1A2000097
:1039C00000E100E0FF00FFFF0844FF1F8C56FF1FCF
:1039D0000854FF1F90B8001114F00040FF7FF8FF5B
:1039E000FFFF9FFF0080FF1F006FFF1F3B000108CC
:1039F000002210B51100112007F04AFC10BD000094
:103A0000F8B500230926374F374C3B62E368112095
:103A1000B343E36007F0F4FC112007F0A9FE112086
:103A200007F0C6FC402322688025134323608023CF
:103A30006268DB0213436360A3682C4A2B43A360D4
:103A4000A36802211340A3608023A2689B01134353
:103A50001022A360236C072093432364236C0F3A46
:103A60001343236480235B003B62226B204B1A408C
:103A70002263626B1A406263A26B1A40A263E26B1C
:103A80001340E363E3681B4A1340E36006F0F4F974
:103A90000121072006F004FB174B11205A6C154337
:103AA0005D6407F095FDFD21144B154A89005A50BD
:103AB0008023C720626B5B0313436363E36880006A
:103AC0003343E3600F4B104A195811408022120211
:103AD0000A431A50802292051A6008220B4B5A633F
:103AE000F8BDC04600F000403CF00040FFFFDFFFA3
:103AF000EFFFEFFFFFFF7FFF003800400000FF1FD8
:103B00005118FF1F00E100E0FF00FFFF000005402B
:103B100070B5284C238C002B23D0228A002A21D177
:103B2000DA0023826382A382E38223836383A383F5
:103B3000E38322606260A260E2601F4D1F4A64203E
:103B4000EB8093420AD8FA220020D200934205D992
:103B50001B4A0A21981807F0F3FDC0B2002328720F
:103B6000238470BD0720E11CCA7F01320240CA775E
:103B700005D10325201DC17F01312940C1770832BD
:103B80005200A352002321001A00088A01321B1898
:103B90000231082AF9D1221DD27F9200A350626817
:103BA00023689B18A2689B18E2689B185B099BB26C
:103BB000C3E7C0460461FF1FAC61FF1FB70B0000E5
:103BC00030F8FFFF30B503A804880B20002C0ED17D
:103BD0004968074D08784978090201430A20A9423B
:103BE00005D1012120001980024B1B7A137030BDD2
:103BF000192A0000AC61FF1FF7B5150008AA168846
:103C00004A680F4F14785278120222430A24BA42AB
:103C100014D10122DBB2019200962A0007F0A8FA23
:103C2000041E0BD1074B1B68002B07D068782A783D
:103C30000002104342425041013098472000FEBD2F
:103C4000022900003061FF1F30B50125037904000F
:103C5000BFB02B4211D00A49408806F0F5FD28423A
:103C60000BD0084B01A95B8D4D800B80064B0022C9
:103C70001B7A60880B7103F0C7FE3FB030BDC046B1
:103C80002861FF1F4840FF1FAC61FF1F10B50549A9
:103C9000054806F08FFD0421044A054806F04CFD56
:103CA00010BDC0462861FF1FFFFF0000BCB8001117
:103CB0004840FF1F10B5024804F028FD10BDC04663
:103CC000493C0011012303700B4B1A7A4270022207
:103CD00082709A78C270DA780271032242711A797E
:103CE00082715A79C2710C2202729A794272DB791E
:103CF00083720B207047C046AC61FF1F022310B5D2
:103D00000370013B43700533837010330371443BF0
:103D100043712A3383714433C37100230372064B0A
:103D200004001B8843720A30FFF7CCFF831D0A3062
:103D3000C0B2E37010BDC046AC61FF1F10B51420C7
:103D400007F016FB124B14220021186007F038FD13
:103D5000002007F025FB012007F072FB022007F08E
:103D60009FFA032003F076FF042005F08BFF052067
:103D700003F0B4F9062003F081FE072001F018FAE1
:103D8000082006F0B9FC092000F0EAFF10BDC0468B
:103D90003461FF1F07F0C4FB012007F0D1FA07F0E0
:103DA00027FB0000094B10B50400984205D00129FB
:103DB00004D12000064906F0FDFC10BD0229FCD10B
:103DC000013904F061FC0028F3D0F6E7FEFF0000A3
:103DD0005A61FF1F70B50D7A100004AA2C001688D6
:103DE00010221440154220D1002E20D10A78022A38
:103DF00018D14A68517815780E4A09022943914230
:103E000005D00D4A914209D01C800A2404E01422F6
:103E10000A491A8007F0DCFA200070BD0C2208491C
:103E20001A80F7E71C800124F6E70824F4E70B2446
:103E3000F2E7C046F3FF0000F4FF00009042FF1FCE
:103E4000A8B9001110B504000749084806F0B2FCF3
:103E5000074804F09BFB0020E40704D50721054A2E
:103E6000054806F069FC10BD5A61FF1FFFFF000006
:103E7000A53D001100B900118C40FF1F00B50C4B8F
:103E8000BFB01A780B4902A800F096FC6B4680B2CE
:103E9000D880002809D06A46074B01A91B88938067
:103EA000064B0022188803F0AFFD3FB000BDC046AE
:103EB0003861FF1F3961FF1FE640FF1FF041FF1F00
:103EC00000B50C4BBFB01A780B4902A801F0E2FC18
:103ED0006B4680B2D880002809D06A46074B01A9FA
:103EE0005B8D9380064B0022188803F08DFD3FB058
:103EF00000BDC0466261FF1F6361FF1F8C40FF1F52
:103F0000F041FF1FF7B50E00377A1C0008AB110017
:103F10003D001A8820231D401F423CD13378022BDC
:103F20003BD173681F785B781B023B431E4FBB423B
:103F300008D01E4FBB4214D01D4DAB4221D00A25E4
:103F40002800FEBD002A2AD1142C2AD82200F068AD
:103F500007F03EFA174B1C70012CF1D9FFF7B0FFA8
:103F6000EEE7002A1BD1202C1BD82200F06807F0B6
:103F70002FFA114B04211C70104B187807F040FBEE
:103F8000DEE7E3B20124009201940A00310007F059
:103F9000EFF80500D4E70825D2E70125D0E70B2587
:103FA000CEE70D25CCE7C046F3FF0000F4FF00008C
:103FB000022900006261FF1F3861FF1FE461FF1FDB
:103FC000332310B5040003700A220749013007F0BB
:103FD000FFF9064B0F201B681A0AE37222731A0CB2
:103FE0001B0E6273A37310BDAC61FF1FD461FF1F72
:103FF00030B5012503790400BFB02B4213D00B4923
:10400000408806F021FC28420DD06A46084B02A8E1
:104010001B889380FFF7D4FF6B46D880002260880E
:1040200001A903F0F1FC3FB030BDC0465A61FF1F4B
:10403000E640FF1F10B5024804F068FB10BDC04603
:10404000F13F001170B5160004AA148805AA15786E
:104050004A685078117800022A4A084380180528D7
:104060004BD807F01DFB03131E29343F0720042CF7
:104070000BD80522121BAA4200D92A0022491A8015
:104080003000091907F0A4F9002070BD0720112C99
:10409000FBD81222121BAA4200D92A001B491A80FF
:1040A000EEE707200E2CF0D80F22121BAA4200D9EF
:1040B0002A0017491A80E3E70720032CE5D80422D9
:1040C000121BAA4200D92A0012491A80D8E70720F9
:1040D000032CDAD80422121BAA4200D92A000E4966
:1040E0001A80CDE70720032CCFD80422121BAA4246
:1040F00000D92A0009491A80C2E700220A201A8042
:10410000C3E7C046DCD5FFFF4BB900118061FF1F3C
:104110003BB9001136B9001131B900112CB90011A9
:1041200010B50D21024A034806F006FB10BDC0463B
:1041300020B90011FC40FF1F13B5104C0423217C53
:1041400001AA00F061F9002815D16B469A8823680E
:1041500052BA92B25343228909491B0C9B184B80D7
:104160006B46DA88636852BA92B2534362891B0C79
:104170009B188B8016BD0120FCE7C0469461FF1F91
:10418000AC61FF1F37B5174C07236A46217C00F04E
:104190003BF9002824D16B461B787F2B20D86B4637
:1041A000DD78F0232A041B031A406B469B880E49D6
:1041B0005BBA9BB21A4323682D09534322891B0C17
:1041C0009B184B806B465A789B7812031B011A434D
:1041D00063682A43534362891B0C9B188B803EBD46
:1041E0000120FCE79461FF1FAC61FF1F7FB5022631
:1041F000154C0022217C03AB0096050000F0D6F898
:10420000002802D0012004B070BD0E23217C0122C1
:10421000280000966B4400F0C9F80028F2D16B46E4
:104220009A892368D2BA5343228908491B149B18E0
:104230004B806B46DA89636852BA92B25343628903
:104240001B0C9B188B80DEE79461FF1FAC61FF1F86
:1042500070B5114C237C002B0FD0382B0ED10F4D95
:10426000280000F051F8CC23AC222800217C9B01CF
:1042700000F012F9280000F085F870BD084BE289C3
:104280009A42FAD1054D280000F03EF8002228009D
:10429000217C00F0E3F8EDE79461FF1FD441FF1F9C
:1042A0008305000070B5144C237C002B1FD063697C
:1042B000002B1CD0114D280000F026F8636928005F
:1042C00098470400280000F05DF8002C10D10C4B3A
:1042D0000422995E002905DA9C801A8801321A802E
:1042E000200070BD074A9142F7DD9A80F5E701246E
:1042F000FEF786FEF4E7C0469461FF1FD441FF1F1E
:10430000AC61FF1F0F27000070B5C17905000C00DC
:10431000631E9C411A4BE402E41849000460C9B2D0
:10432000007905F0F3FEE979687949000131C9B2F5
:1043300005F0ECFEE8790930C0B207F039F8002347
:10434000E36661332360AA795B3B002A0ED02268C2
:104350009A43023B134323600A23E361073323623A
:1043600000232363A3630133E36370BD22689A4390
:10437000022313432360462363610633A361EFE7FF
:104380000050004070B5002504000368DD66C07968
:104390000930C0B207F034F82900207905F052FE48
:1043A0002900607905F04EFE70BD0000F8B51E00D2
:1043B00006AB1D78002304681700E366616007F010
:1043C00067F801238022E3662B0027615200013B3E
:1043D00008D206F0DDFF08200A4A1168002D03D13B
:1043E0002800F8BD2261F2E7236F034203D023695E
:1043F000013D3370013613685B1A032BEED901259A
:10440000EEE7C0466008FF1F70B51C00002305687A
:104410001600EB66696007F03BF801238022EB662B
:1044200023005200013B08D206F0B2FF08200A4ADE
:104430001168002C03D1200070BD2A61F2E72B6FB8
:10444000034203D02B69013C3370013613685B1AB9
:10445000032BEED90124EEE76008FF1F002370B59F
:1044600004681500E366616007F012F80123E36653
:10447000256106F08DFF8020064A80001168636B7D
:10448000034205D113685B1A032BF8D9012070BDD4
:104490000020FCE76008FF1F70B51D0000230468C2
:1044A0001600E366616006F0F3FF0123E366266110
:1044B0000F33626B1A42FCD02B0A23611023626B0C
:1044C0001A42FCD0EDB2256106F062FF8020074A57
:1044D00080001168636B034205D113685B1A032BDC
:1044E000F8D9012070BD0020FCE7C0466008FF1F1E
:1044F00010B5084CE368002B08D18022064B52020D
:104500001B689B186360054B1B68236006F068FFFF
:10451000A06010BDD461FF1FC8F00040CCF0004087
:1045200070B5184A936A916A9942FBD116498A6814
:104530009A421FD39A1A8B60144B0126186893B2C3
:10454000D202D20E4343424300204C681B0A1B197F
:1045500012029B180E4C0A684B60551CA3420CD8E3
:10456000002801D04B600A600A4A136008680A4BB1
:10457000186070BD581E821ADDE7084A30009B188B
:104580002A00EAE700F00040D461FF1F140AFF1F71
:1045900040420F00C8F00040CCF00040C0BDF0FF2A
:1045A00070B51F4C23793F2B01D93F2323711D4B3D
:1045B00022791A701878C0B206F09AFE18231A49A8
:1045C0001A4A0B801A4913800B805380A37919492A
:1045D00080200B800C21938001334B43164D191C16
:1045E0000001834200D9011C2980D1806379002B0E
:1045F00011D101336371237A012B01D80223237275
:104600006279237A0D4853430A21584307F098F8FA
:104610000B4D286070BDA02BEDD9A023EAE7C04662
:10462000C861FF1F480AFF1FEE41FF1FB043FF1F75
:10463000EC41FF1FEA41FF1FE841FF1F710200002C
:10464000B861FF1FF8B519210020FEF7CFFE114C0D
:10465000011E114D09D10C22104BC1CBC1C4280041
:1046600007F0AEF8FFF79CFFF8BD0C2220000C49C4
:10467000FEF790FE0C2802D0084B43CB43C40C221B
:1046800028000849FEF786FE0C28EBD00C220021FA
:10469000E5E7C046C861FF1F9461FF1F9CB9001188
:1046A000FC0C0000F50C0000F0B51D4C8022A54468
:1046B0000400882069465201400506F0E1FF90227F
:1046C00012016A441300200032C832C316C816C350
:1046D0008023144C144FA6689B033343A3603B60B4
:1046E00006F0AEFD8823A0685B05C01806F0F0FD5B
:1046F0000025882329008022A0685B05C018401986
:104700006944520006F02CFE80230135FF355B0121
:104710009D42EED1A6603E60044B9D44F0BDC04674
:10472000FCEFFFFF2043FF1F9808FF1F041000004D
:10473000F0B5040087B0002825D0684606F018FFC1
:104740001B4C022806D106226946200006F090FD87
:10475000002816D06946002301250F262F00E25CB1
:10476000013310091030874038002F003240974045
:104770003A0002434A610439062BEFD16846FFF73D
:1047800093FF07B0F0BD182269460A4806F078FF8B
:104790006A46A300D358013305D01822FF2168468A
:1047A00007F00EF8EAE70134062CF1D1E9E7C0463C
:1047B0006509FF1F00090011F0B5002504000E0077
:1047C00085B0AA4200D183E04B1C087801934B7856
:1047D0008978377909021943F3783F061B040B43A4
:1047E0001F43039720706570252800D193E033D8CC
:1047F000112813D806F084FD66000D010D010D018E
:104800000D01A700B500AE000D010D010D010D0158
:104810000D010D010D010D01E7000701232800D155
:10482000C0E0DB2800D016E1042A00D8A9E010255A
:10483000052A05D0551F2A003800711D06F0C8FD55
:1048400005223100200006F0C3FD2A003900601D5A
:1048500006F0BEFD05353BE0562856D010D833286B
:1048600000D19AE0552836D02628DAD1894B290084
:10487000132218001D0006F0A3FFFEF7C1FB59E04C
:10488000712800D174E0722800D17DE0DC28C8D105
:10489000022A00D875E07378BFB26370B378A37052
:1048A000032A05D0033A390092B2F01CFEF7ACFCA3
:1048B00010223900E01CFEF76DFDC51C002807DA48
:1048C00060705CE00C222000734906F081FD0C252D
:1048D000280005B0F0BD013A704D0C2A13D8002A0B
:1048E0000AD02800019906F073FDFFF759FE0C224B
:1048F00028006B49FEF788FC29000C22601C06F09A
:1049000067FD0D25E4E70C22EBE7644D654B2A00BB
:1049100043CB43C2E9E7013A5E4D0C2A11D8002A85
:1049200008D00199280006F053FD0C2228005E49AA
:10493000FEF76AFC29001322601C06F049FD1425CD
:10494000C6E70C22EDE706225849601C06F040FD40
:104950000625BDE712225649601C06F039FD1325D5
:10496000B6E708225349601C06F032FD0925AFE77F
:104970007178F02905D8504B188801F0E7FB022523
:10498000A6E7FF236370FAE74C4B012A03D0727845
:104990005A706270F3E75B78F4E72000FFF710FBD2
:1049A000050095E7042A04D9454D2F6006F018FD4F
:1049B000A860FFF7B5FD0422039003A9601C06F070
:1049C00007FD052584E73F4D062A15D90622280054
:1049D000019906F04DFC00280ED00622019928000E
:1049E00006F0F6FC062238492800FEF70DFC0123EC
:1049F000324A51780B43537029000622601C06F09E
:104A0000E7FC072564E7012ABBD07078FFF790FE2A
:104A1000B5E7012800D004E7931E2C4F132B06D8CE
:104A20007378002B0BD100F009F900F03FF9284B07
:104A300039001D78601C6A1E06F0CAFC48E7551E46
:104A40002A000199380006F0C3FC38002149AAB2B7
:104A5000FEF7DAFBE9E7DA2893D1042A91D9082A8C
:104A600015D9B37972791B021343F27912041A43F0
:104A7000337A1B0613433B603B680522310020005C
:104A8000039306F0A5FC0422601D03A96CE7FE2336
:104A90006370F1E79461FF1FA8B90011C861FF1F9F
:104AA000FC0C00009CB90011F50C0000A061FF1F78
:104AB0008061FF1F2443FF1FF041FF1FC461FF1FE0
:104AC000D461FF1F6509FF1FADAC0000C563FF1F68
:104AD000C363FF1FAEDE000070470000020010B588
:104AE000094B0A32094C92B2DA815A8298811882B3
:104AF000207802F091F90422054B012120781A70E8
:104B000006F07EFD10BDC046AE42FF1F0E64FF1FC3
:104B10000D64FF1F013870B5042809D806F0C0FDE8
:104B20000309230812001E4B0221187806F068FDC5
:104B300070BD1B4B0821187806F032FE0022194B7D
:104B40001A72F5E780220024164B154D52001A8187
:104B5000082128781A68DC7206F082FD2100287886
:104B600006F0AEFCE4E70E4B0821187806F018FEBC
:104B70000D48FFF7C3F80D4B0D4A9B7993800D4A02
:104B800013800022074BDA720132FF321A810A4B7E
:104B90005B78002BCCD0094A136006F029FDC7E7EB
:104BA000E461FF1FB861FF1FF941FF1FC861FF1FCC
:104BB000B043FF1FEA41FF1FC461FF1F34F00040F4
:104BC00010B5002905D1082803D10131013005F0C5
:104BD00067FA10BD10B501290FD108280DD10021A9
:104BE000013005F05DFA054B1B78002B05D026221D
:104BF000034B04485A72FFF771FF10BDE663FF1FB5
:104C0000B861FF1FC40900000300F0B50A4D8E18FB
:104C1000B14202D152008018F0BD0C782F682409EF
:104C20003C5D0F271C700C7801313C402F683C5DC7
:104C30005C700233ECE7C046E441FF1F0E22124BCA
:104C400010B51A700D23114C11492370093A043B19
:104C50001048637006F0BCFB2D2301220E490F485B
:104C6000E371FFF7D1FF01220D49FFF7CDFF0122CC
:104C70000C49FFF7C9FF030000200B490200187020
:104C8000FEF7C2FA10BDC046E263FF1FC363FF1FF9
:104C90004BB90011C563FF1F6709FF1FCB63FF1FDF
:104CA0006609FF1F6509FF1FAEDE000070B5134CDB
:104CB000142220001249FEF76DFB431E114D132BE9
:104CC00019D8AB78002B16D0431C2B7009236B70BE
:104CD00000230019037028780B4B01302900C0B263
:104CE000187006F0EDFC297822000139C9B20020C5
:104CF00005F040FC70BDFFF7A1FFECE7C563FF1FA7
:104D0000AEDE0000C363FF1FE263FF1F10B5114B4F
:104D10001A781870002A0ED000280BD10E4B1A7882
:104D2000062A07D85423D340DB0703D50B4B18784A
:104D300002F072F810BD0028FCD0074B1B78012B45
:104D400002D0033B022BF5D8044B0121187806F062
:104D500057FCEFE7E663FF1F0D64FF1F0E64FF1FA4
:104D600070B5504E504A51493070082005F08EFA07
:104D70000121092005F094F9092005F075FA0121B7
:104D8000002005F08DF9002005F06EFAFEF738F9E5
:104D900006F0AEFC032246494648FFF735FF2D24B6
:104DA000030004221C7044490130FFF72DFF30231B
:104DB0000470424D424C437083702E3B062220000B
:104DC0004049EB87FEF7E6FA062813D0200006F0EC
:104DD000CFFB022809D00321200006F029FC8D23F7
:104DE000E3706E3B2371193363710622200035494D
:104DF000FEF70AFA344B1B68FC335C64FFF756FF7E
:104E00000020FFF783FF314C314A0121314B1278EA
:104E1000207801F0C3FF304A304B1278002120780F
:104E200001F0BCFF01222E4B1A702E4B9B78552BA4
:104E300031D12D4B3B325A722C4B2D4AAB81EA813A
:104E40002B826A822021307806F0EAFA0120404263
:104E500005F0DCFB0120404205F078FCFFF760F92B
:104E6000FEF714FF00F0AEFC01204042FEF7EAFF1F
:104E7000012006F0BDFCF02001F04CF90121307852
:104E800006F0BEFB307802F023F91A4806F080FBEA
:104E9000FEF7B6FD70BD6422174B5B7953431A00D1
:104EA0000A32CBE7E461FF1FC14B0011D54B001163
:104EB0002443FF1F8061FF1FA061FF1FAE42FF1F41
:104EC0006509FF1FADAC00003064FF1F0E64FF1FBB
:104ED0001842FF1FF941FF1FE263FF1FC363FF1F5B
:104EE000B463FF1FC461FF1FB861FF1FC409000046
:104EF000CE090000E661FF1FC861FF1FF8B50A0078
:104F000020230D001A4019425DD05C4B1B78002B0A
:104F100042D0FFF705FB5A4B5A4C5B4E99686268CA
:104F2000737A8A1ADB039A4202D36160FEF768FD46
:104F3000327A217A531EDBB2994230D1FFF788F9D9
:104F4000637A002B25D0013BDBB26372002B20D1AA
:104F50004E4B9B78552B01D106F04AFBE37A002B90
:104F600012D00023A27AE3729A4202D0A372FEF713
:104F7000CFFD474A474F1388380001331380FEF7AF
:104F8000BDFE390006F0BCFA642370795843FFF780
:104F9000A5FD237A0133237220206840F8BD914299
:104FA000CED300272772FFF77DF9A37ABB4202D048
:104FB000A772FEF7ADFD374F3800FEF79FFE3900B0
:104FC00006F09EFABCE70BB2002B0ADA324B1878D7
:104FD00006F04EFA002801D006F01AFA80200002EE
:104FE000DBE70224214206D0264B01201A72FFF78C
:104FF0008DFE2000D1E70B071BD5FFF791FA204B60
:105000002049214C98684A68637A821ADB039A42E5
:1050100002D34860FEF7F4FCFFF744F9FFF718F9F4
:1050200000F0EAFB2368DB0701D5FFF703F808204F
:10503000B3E710230E001E40194209D0FEF768FDA9
:105040000E4B1B78002B01D1FEF734FE1020A4E795
:105050000124214209D0114800F06EF806F040FA10
:105060003100092005F01CF8C3E7042408002040A3
:10507000214200D192E7FEF701FFBAE7E663FF1F86
:10508000D461FF1FB861FF1FC861FF1FC461FF1F0C
:10509000AC61FF1FF941FF1FE461FF1FDC41FF1FEF
:1050A000F0B51B4B1B4F1B883A8804001A4E1B4D52
:1050B00085B09A420DD832889A420AD3184B1A8882
:1050C0002B889A4205D1174A174B12881B889A429F
:1050D0001BD0052001F074F83B8802AA13803388A6
:1050E000019053802B88114D93800F4B02A91B8890
:1050F000D3800F4B2A78188802F090FD0D4B0821C1
:105100002878019A1C7006F003FA05B0F0BDC0467D
:10511000B263FF1FEE41FF1FEC41FF1FEA41FF1F7B
:10512000B063FF1FAE63FF1FE841FF1F0E64FF1F48
:10513000F041FF1FAC63FF1F13B50C4B1C78002C14
:1051400011D1002801D00A4B18600A4A0A4B117885
:105150000A4A10780A4A01920A4A0092002205F08F
:1051600001F9200016BD1124FBE7C0460D64FF1FA6
:10517000A863FF1F0C64FF1FFC63FF1F0E64FF1F6B
:10518000E863FF1FEC63FF1F10B5064B12201B786E
:10519000052B06D1044B13221988044B187801F013
:1051A000EBF910BD0D64FF1FF041FF1F0E64FF1FE0
:1051B00010B500240122114B52421870104B1C7084
:1051C000104B1A8001F084FF04220F4B21001A704B
:1051D0000E480C3206F09CFA102221000C4806F012
:1051E00097FA07220B4B1C600B4B1C700B4B1C706F
:1051F0000B4B1A700B4B1C7010BDC0460E64FF1F8A
:105200000D64FF1FF041FF1F0C64FF1FFC63FF1FB5
:10521000EC63FF1FE863FF1FC263FF1FC163FF1F33
:10522000F241FF1FC063FF1FF8B5174C0600257839
:1052300006A814240078052D23D1B41F134FA5B25E
:105240001824BD421DD88D1FADB2BD4219D8FA2514
:105250006D00AA4215D21D000D4F0A3DADB2BD42F0
:105260000FD80C4C26800C4C21800C4900240A805D
:105270000B4A1380FFF714FF0A4B0421187806F03D
:105280008FFA2000F8BDC0460D64FF1F790C0000A6
:10529000750C0000EE41FF1FEC41FF1FEA41FF1FAC
:1052A000E841FF1F0E64FF1FF0B50BB20D0089B07F
:1052B000002B00DB70E1A44E307806F0D9F8041E14
:1052C00050D00378A22B00D122E1D02B1AD0912B01
:1052D00045D143780E2B42D19C4B82889A423ED1D5
:1052E0009B4A83681278052A39D1032018567F28F3
:1052F00035D0984B1B68002B31D05B68002B2ED02B
:1053000098472CE08078072829D806F0C9F90428A6
:10531000183F3F74A8D86378002B0CD101218C4B27
:1053200019708D4B1A78002A5BD08C4B307801F0C5
:1053300035FD002855D00722854B1A7051E0617861
:105340000029F8D1E378002B11D0854A854B1278DB
:10535000307801F023FD60706378002BEBD12000E2
:1053600006F056F880200002684009B0F0BD784B86
:105370001B78022BF3D00121307806F079F9002850
:10538000EAD10121307806F03BF9E5E76378002B9C
:10539000D1D16F4F032807D13B78052B02D10133C0
:1053A0003B701EE00223FBE76F4B1A886F4B0293A2
:1053B000002A0BD01B78002B03D00121307806F097
:1053C000A7F83B78062B04D1013BE9E7029B1A7052
:1053D000F7E7042B41D10121029B3078197006F0C8
:1053E0000FF95C4B1B68002BB9D01B68002BB6D0A3
:1053F000574A107884E76378554F002B27D106224F
:10540000211D5B4805F0E4FF62895A4B5A491A8016
:10541000A2895A4B1A80E3890B80052139705849BB
:105420000A80584A1380228A574B1A80574B1B78A0
:10543000012B09D11F2000F0C3FEFA229200424343
:105440000421307806F064F80022484B75E7312BD0
:1054500000D070E70022454B1A700323A0E7062214
:105460000021434806F054F90023454A04211380E3
:10547000444A30781380444A138006F091F9082199
:10548000307806F08DF9A379083B5A425341304AEF
:1054900003331370304B1B78002B06D0334B30781E
:1054A0001A78002A06D001F0B7FC0122314B524293
:1054B0001A8096E70121197006F0A2F8F5E7082195
:1054C000307806F06DF96378002B00D047E72C4B5D
:1054D0002D4F0293E388029A04211380294B3078E0
:1054E00003932389039A138063893B8006F0C0F8F5
:1054F000002800D033E7264B1B68002B00D12EE795
:10550000039902983A88098800881B68984726E71B
:105510004379132B00D022E70389012B0AD11D4BBD
:105520001B78022B06D10821307806F039F9FFF7F5
:105530002BFE14E7052000F043FE0821020030781E
:1055400005F0E6FF0BE7C0460E64FF1F05140000E0
:105550000D64FF1FA863FF1F1842FF1FF941FF1FC3
:10556000E263FF1FC363FF1FE463FF1FE663FF1FC8
:10557000B563FF1FF041FF1FBC63FF1FBE63FF1F2A
:10558000B263FF1FB063FF1FAE63FF1FB463FF1F53
:10559000A463FF1FAC63FF1F8020C001014200D045
:1055A000E2E6CB0731D5324B1B78002B1DD0314EB4
:1055B00005AC3378052B1AD1023B23702E4B21000A
:1055C0001B7823722D4B1B7863722D4B187801F0DA
:1055D00089FB002809D007202A4B30701B68002B5C
:1055E00003D01B68002B00D098470120BCE60E209A
:1055F000254B06221B7825492370254B1B786370A9
:1056000002ABC01805F0E4FED8E7022308001840FA
:10561000194209D0174B1B78052B03D11D4B188855
:1056200006F0FEF802209FE60424214203D0FFF793
:1056300037FD200098E6082308001840194200D1E1
:1056400093E6154B1C78012C03D0022C0DD00820BA
:105650008AE6124B124A134913481B88128809889C
:1056600000880094FFF7E0FDF1E7FFF78DFDEEE71E
:10567000E663FF1F0D64FF1FF241FF1FC063FF1FA2
:105680000E64FF1FA863FF1FC263FF1FF341FF1FCC
:10569000C163FF1FF041FF1FAC63FF1FE841FF1F05
:1056A000EA41FF1FEC41FF1FEE41FF1F10B502A8AA
:1056B00004880B20002C10D1496808784978090229
:1056C00001430C48814209D1022119800A4B5988B3
:1056D0001170DB7800205BB2537010BD074C0A20BC
:1056E000A142FAD102211980034B998811705B798C
:1056F000F0E7C0466E2A0000AC61FF1F6F2A000071
:10570000F7B5150008AA16884A680F4F1478527822
:10571000120222430A24BA4214D10122DBB20192BE
:1057200000962A0005F024FD041E0BD1074B1B68D0
:10573000002B07D068782A7800021043424250417B
:10574000013098472000FEBD022900002064FF1FA1
:1057500030B5012503790400BFB02B4225D0144990
:10576000408805F071F828420CD0124B01A95B8DDE
:1057700000220B8002234B800F4B5B888B8060885C
:1057800002F042F90D49608805F05EF8C0070CD5BB
:105790000B4B01A91B8800220B8002234B80064B78
:1057A0009B888B80608802F02FF93FB030BDC046E7
:1057B0001864FF1F1C42FF1FAC61FF1F1064FF1F16
:1057C0007642FF1F10B5074C0749200004F0F2FF96
:1057D0002000064904F0EEFF0721054A054804F0C1
:1057E000ABFF10BDFFFF00001864FF1F1064FF1F18
:1057F000C8B900111C42FF1F10B5024802F086FF15
:1058000010BDC046515700110200F0B501270A48EB
:105810000A4E51188B1A002B00DCF0BD08241578B5
:105820004308684038404000805B013C58406D08A8
:10583000002CF5D10132EDE7FFFF0000E2B90011C5
:10584000F0B500250F269D4200DBF0BD4C5D070939
:1058500044403440A400A05801357840F3E70000EC
:10586000F0B589B06A460D000B000F271100103506
:105870001C780133260024093E4016705470023211
:10588000AB42F5D12023024AFFF7DAFF09B0F0BDA1
:10589000E8B90011F0B54E780B7889B036020C00EB
:1058A000170001901E43012A61D9954B9E4200D8F2
:1058B00077E001339E421CD1062A17D1CA788B7833
:1058C00012021A430B791B0413434A7912061A4336
:1058D0008C4B5A6100221A705A808B4A5A608B4A4C
:1058E0009A608B4ADA60002009B0F0BD8822520528
:1058F000EEE7884B9E423CD182498B78002B00D04A
:10590000F6E00C2A31D10F22A3789343E2781202F9
:1059100013432279120413436279120613434B6036
:10592000E279A07912020243207A00041043627ADD
:1059300012060243CA60E27AA07A12020243764853
:105940004A81834208D804236E49142201980B70BF
:1059500005F03EFD1420C7E71201D21889235B052C
:105960009A42F0D801238B70BDE7022AFAD00523B2
:10597000EAE76A4A01239642E6D1FFF705FC052FC4
:105980000CD9E378A2781B021343227912041A433C
:1059900063791B061343624A0393136005F028FEE4
:1059A000A1E7584D2B78002B9DD1AB78002B00D16F
:1059B000A0E02B8901339BB20093B34200D091E069
:1059C000132AD4D9CF7C8B7C3F02122120001F43A5
:1059D000FFF71AFF874200D08EE0002E3DD1E3781A
:1059E000A2781B0213432279E96812041A436379EF
:1059F0001B06134303930A228B4212D1FF23A37089
:105A0000E370237163716B89002B09D1E37B227CE6
:105A10001B0212041343A27B13431B0901336B8146
:105A200000226B89002B8ED0002A67D1686837016D
:105A30003818000B6B6900030390984205D9686120
:105A400005F046FCEB780133EB7068681022A11C6E
:105A5000381805F085FC2E8145E76F89009A7B1E7A
:105A60009BB293423AD1E278A37812021A43237987
:105A700005A81B04134362796C6812061A43EB688D
:105A800000920392211D0C22049305F0A1FC012039
:105A9000260004A940421036FFF7E2FE013F012F25
:105AA00017D1009A0B232861824200D04CE70422D0
:105AB0001C49200005F054FC042203A9686805F085
:105AC000DFFDE968039AFF23914200D13CE7F73BF1
:105AD0003AE73100FFF7C4FE1036DFE70923B7428B
:105AE000A4D831E7009BB34200D9FCE607232BE79B
:105AF000022329E7032327E7062325E70A2323E7D1
:105B0000FFFE00009042FF1F00000111FFFF000098
:105B10005048593601FF0000FFFF001102FF00004E
:105B200034F000409C42FF1F10B5034C0B000122D3
:105B3000210000F06BFA10BDE95C00110B8870B514
:105B400006000D000224162B11D92B00032209494F
:105B500000F05CFA041E0AD1074B2A881B88191C26
:105B6000934200D9111C300089B200F0EFFA2000F6
:105B700070BDC046155D00113664FF1F10B54A7830
:105B80000400013A0B000220012A07D80A78002AF3
:105B900004D005222000024900F038FA10BDC046AA
:105BA000435D00110A7810B50B0004000220002AA2
:105BB00004D007222000024900F028FA10BDC04698
:105BC000EF5D00110A7810B50B0004000220002AD6
:105BD00004D009222000024900F018FA10BDC04686
:105BE000555E001110B5034C0B000B22210000F094
:105BF0000DFA10BD855E001110B5034C0B000D228F
:105C0000210000F003FA10BDF75E001110B5034C3F
:105C10000B000F22210000F0F9F910BD515F0011B7
:105C20000A7810B50B0004000220002A04D01122CB
:105C30002000024900F0EAF910BDC046615F001182
:105C4000002310B51322190000F0E0F910BD000088
:105C500010B5034C0B001722210000F0D7F910BD3E
:105C6000B35F0011002310B51922190000F0CEF91E
:105C700010BD000010B5034C0B001B22210000F0EA
:105C8000C5F910BDED5F0011F7B584890D00060060
:105C90000121002C22D000238268D3561778002BD4
:105CA0001EDA0C2C1AD90C3CA4B2131940880093AC
:105CB000230002F086FE431E984101307B06DB0F75
:105CC0006B703F23013C1F40A4B22870AF70AC80C2
:105CD000002C07D0B3680133AB6000210800FEBD83
:105CE0000020EBE7AC60F8E70B7803704B8843705B
:105CF0004B881B0A83700B79C37004207047042003
:105D0000022B06D10020537811781B02009A0B4316
:105D1000138070470B8803700B881B0A43700220A6
:105D200070470420009983420AD1537810781B02EF
:105D300003430B80D37890781B02034300204B80F1
:105D40007047F8B50D004B7801240021461C037004
:105D50002B788B4201D82000F8BD6B78B01C4F1C0B
:105D6000012B10D1890069184B88022233704B88AF
:105D7000B9001B0A7370691805F05AFB0436043425
:105D8000A4B2F9B2E4E7122359436B185A880431DC
:105D900032705B8810221B0A7370691805F048FB8B
:105DA00012361234ECE770B5049D14001E00052B6A
:105DB00001D8042070BD637812781B0213432B8036
:105DC000E378A2781B02134302226B802A71211D03
:105DD000681D063E05F02CFBB2B22A81E92AE8D8FC
:105DE0002800A11D0A3005F023FB0020E2E7002374
:105DF00010B50A789A4201D8900010BD9A008A180E
:105E00005488013304705488DBB2240A44709488A7
:105E100084709288120AC2700430EAE710B511004B
:105E2000029C062B04D004201022142B01D010BD9C
:105E3000022222714B7808781B0203432380CB781F
:105E400088781B02034363800431601D05F0F0FA7B
:105E50000020ECE710B50C788B7804315C43E4B299
:105E600003702200013005F0E3FA601C10BD04202D
:105E7000022B06D10020537811781B02009A0B43A5
:105E80001380704710B50C000A88023105F0D0FA73
:105E9000208810BD70B504000D0004981100012B7E
:105EA00001D8042070BD1678527812023243028065
:105EB0000200F13255701470E125002C00D10C3530
:105EC000023B9AB24280AA42EBD80231043005F07C
:105ED000AFFA0020E6E70420009983420AD1537804
:105EE00010781B0203430B80D37890781B02034386
:105EF00000204B80704710B50C000A88023105F075
:105F000097FA208810BD000070B501211E00042002
:105F1000049C0E400B4218D1CB40DDB28D4214D907
:105F20000A49DBB2098899420FD32300EE331D7072
:105F30003300580011184978165C090231430133C7
:105F40002152D9B28D42F4D8002070BDA842FF1F63
:105F500010B50C000A88023105F06AFA208810BDDD
:105F600010B50C788B7804315C43E4B203702200E6
:105F7000013005F05DFA601C10BD10B511000298EB
:105F8000032B01D8042010BD14785278043B120270
:105F900022430280CA788C781202224342809AB24D
:105FA0008280EB2AEED80431063005F041FA002059
:105FB000E9E710B50C000B8803700B881B0A4370CF
:105FC0004B8883704B881B0AC3708A880430063163
:105FD00005F02EFAA088043080B210BD0420012BF9
:105FE00003D100201378009A1370704710B50C008D
:105FF0000B8803700B881B0A43704A8802300431F7
:1060000005F016FA6088023080B210BDF0B589B094
:1060100003931E4B029242000700D05A019102F0F6
:1060200020F81325061E2DD0029B01240370019B2E
:10603000002B04D0001903999847001984B26B46CD
:106040001B7A5BB2002B0FDA1021380002F01CFB28
:106050001925002813D130003219E1B202F066FC94
:10606000051E0CD10C34A4B2042304AA380005A9DF
:1060700093800696948101F0AFFD051E02D030009A
:1060800005F006FB280009B0F0BDC0463464FF1FD0
:1060900070B505000C0000280CD00020814209D00A
:1060A00010222000044905F0C3F901202B78237346
:1060B0006B78637370BDC04628BA0011F0B5060056
:1060C0000D0017001C0085B002291BD000201029EC
:1060D00007D1022B07D0102B03D115E00020102C84
:1060E00008D005B0F0BD69463800FFF7D1FF2A009F
:1060F00069460BE069463000FFF7CAFF2200694697
:10610000380004E0022BE9D12A003900300005F004
:10611000FFF8E6E7031CF02800D9F0230320084924
:106120009AB2013A0B80D317034006499B189B1083
:106130000B80D30F04499B185B100B807047C0463F
:10614000AC42FF1FAA42FF1FA842FF1F034B1B8840
:106150008B4202D3024B4000C1527047AC42FF1F3A
:106160003464FF1F014B4000185A70473464FF1F0E
:106170001722014B1A8070473464FF1F70B5050069
:106180000E2005F0E5F8041E13D0D0230370002381
:106190000622837007494570033005F049F9064B24
:1061A0002100DA8A62811B7E2373044B187805F084
:1061B000E7FA70BD5064FF1F4064FF1FFC42FF1FE1
:1061C000262803D8024B4000C05A70470148FCE71C
:1061D000AE42FF1FFFFF000070B506000C00094D26
:1061E0001C220021280005F093FA074B1E70074B74
:1061F0001C7005F0ADF90123002801D00023122006
:106200002B7070BD4064FF1FFC42FF1F6164FF1FC5
:1062100070B505000D4C0800E260A160102200215D
:10622000656005F05DF8012803D11021A06802F037
:1062300058FD10220021280005F052F8012803D152
:106240001021606802F04DFD70BDC0464064FF1F24
:1062500070B5041E05D1002903D006220D4805F0B3
:10626000E7F80D4B1D78012D11D1002C05D102222C
:106270001A7005F0B5FA280070BD00221A70074B9D
:106280001B78FF2BF7D02000FFF778FFF3E70025FE
:10629000F1E7C0465064FF1F4064FF1FFC42FF1F30
:1062A000030010B5002801D1002010BD00780B4A72
:1062B000002803D15988D1821B7913761378022BD9
:1062C000F2D10023984200D103331370044B1B78A2
:1062D000FF2B01D0FFF752FF0120E6E74064FF1FCC
:1062E000FC42FF1F002911D000280CD04B79012857
:1062F00003D140225242134303E03F2213400328BC
:1063000002D001204B7170474022F4E70800FAE701
:1063100070B5094D0100287800280BD0074C0622E3
:10632000200005F085F821002878FFF7DBFF20002A
:1063300005F03EF970BDC0466064FF1F3A64FF1F60
:1063400000290AD0012808D13F224B799343C02B62
:1063500003D0403B5A425341981C704770B5174DCB
:1063600006002B78FF2B15D00A2004F0F1FF041E45
:1063700010D0D0230370C83B8370114B11491B7898
:106380004670C3700622043005F052F821002878C8
:1063900005F0F6F90C4B1B78012B0DD10B4B1B684C
:1063A000002B03D09B68002B00D09847084B04219A
:1063B0001878084A05F054F970BDC046FC42FF1F2A
:1063C0006064FF1F3A64FF1F5C64FF1F8864FF1F47
:1063D0008C64FF1F60EA0000014B98687047C0465C
:1063E0004064FF1F014BDB68186870474064FF1F63
:1063F000074B10B5DA68136801331360054B187842
:10640000FF2803D08021C90105F0FAF810BDC0466D
:106410004064FF1FFC42FF1FF7B50E0002F0C8F8F2
:10642000051E1CD00E4B06621F78002F00D1077886
:10643000AB791020019304F08BFF041E0FD0D02302
:106440000380C73B8370019BE91DC37006220430A3
:1064500004F0EEFF21003800E66005F091F9F7BD89
:10646000FA42FF1F014B18787047C0466064FF1F57
:10647000054B002805D1054B1A78054B002A00D1A1
:10648000014B18007047C0465064FF1F6064FF1F37
:106490003A64FF1F014B58687047C0464064FF1FB5
:1064A000024B1868431E9841C0B270476464FF1FD6
:1064B000421E03000120152A03D9FF3B5A425341D3
:1064C000D8B27047F0B51C0000230E0085B00390D1
:1064D00002920B70029A934201D3002019E0E55C0E
:1064E0005A1CD2B2002DF8D0029851198142F4DC26
:1064F0000233DFB2A35C18000193FFF7D9FF002835
:1065000007D0013D019A0399EBB233708A4202D160
:10651000E01905B0F0BDDB19DBB2DBE710B50C000C
:1065200002F09EF803001220002B03D021005888AF
:1065300005F0A6F910BD000070B50E4D840063593A
:10654000002B15D0186A002801D005F0E9F82B5966
:10655000586A002801D005F0E3F82B59986A002802
:1065600001D005F0DDF8285905F0DAF800232B51A9
:1065700070BDC0467064FF1F1C4B70B504000E0058
:10658000150099420AD11A4B1B68002B01D1122029
:1065900070BD1B68002BFAD09847F9E7154B99425C
:1065A00015D1134B1B68002B0AD01B68002B07D09A
:1065B0009847002804D1104B1C70104B1D70E7E762
:1065C00029002000FFF7AAFF0028E1D1F3E7080027
:1065D00001F0EEFF0028DAD003780320A342D7D1E0
:1065E0002900300005F04CF9D2E7C046FEFF00005C
:1065F0006C64FF1FFFFF00006964FF1F6864FF1FDA
:10660000F7B50400808801F0D3FF0025A84203D02D
:106610000578A08802F008F81C4E3378002B1FD0B4
:10662000AB421DD11A4B28001978FFF777FF0028DD
:1066300018D000233370A3790820A778A688019387
:1066400004F086FE011E0DD0D0230370CA3B837078
:10665000019B477086808371280005F091F801E066
:10666000002DE8D1A0880B4B8200D358002B01D01D
:10667000FFF762FF1721A088FFF768FDA08801F0EF
:1066800027FDA08801F0FEFDF7BDC0466964FF1F2D
:106690006864FF1F7064FF1FF0B587B01D000CAB6E
:1066A0001B88070001930DAB1B88142002930EABCF
:1066B0001B88160003930FAB1B880091049310AB4B
:1066C0001B88059304F044FE041E1AD0D0230370E7
:1066D000CB3B47708370C670062229000430002D22
:1066E00011D004F0A5FE019B21006381029B00985C
:1066F000A381039BE381049B2382059BA37405F084
:106700003FF807B0F0BD05F003F8ECE7F7B50093EC
:1067100008AB1B8807000C200D001600019304F045
:1067200017FE041E13D0280001F042FF00280FD0EE
:106730000078D0232370C93BA370009B21002381E4
:10674000019B6770A580E680638105F019F8F7BDAD
:10675000014B1878EDE7C046FC42FF1F13B504005B
:1067600064890389C2888188C0780094FFF7CEFFCE
:1067700013BD000010B5044C2068002803D004F0BD
:10678000CFFF0023236010BD7464FF1FA122F0B56A
:10679000818892004A43384B384F1B6804009B188D
:1067A0009D2292009B18827989B01A603B68002B69
:1067B0005FD01D78324B1B68002B04D05B68002B28
:1067C00001D000209847260008363100E079FFF715
:1067D000B7FD237DE0710200E0780493638A29000D
:1067E0000393238A0293E3890193A38800933300E0
:1067F000FFF752FFE378002B0BD1E289A379A18840
:1068000002920196E27928000092012201F0DAFE5C
:10681000E0703B68002B20D0FFF7ACFF194D2878C3
:1068200000281AD0184B1978FFF778FE002814D0EA
:106830002B78E67808200793A78804F089FD011ECD
:1068400009D0D0230370CA3B46708370878086715D
:10685000079804F095FF00232B701721A088FFF7FD
:1068600075FCA08801F034FCA08801F00BFD09B094
:10687000F0BD064B9DE7C0463409FF1F7464FF1F3F
:106880008864FF1F6964FF1F6864FF1FFC42FF1FCD
:10689000F8B5070008000E0001F08AFE041E18D0AB
:1068A0002620FFF78DFC051E00D12578062004F078
:1068B0004FFD041E0DD00021062204F029FFD02335
:1068C0002370C23B21006770A370A680E8B204F079
:1068D00057FFF8BDF0B585B001930AAB1B780700F0
:1068E00002930BAB1B7808000D000092039301F09C
:1068F0005FFE061E22D0102004F02AFD041E1DD0CB
:106900001022002104F004FF2620FFF759FC002884
:1069100000D13078D0232370C13BA370009B2100AD
:106920002372019B67706372029BA580A372039B15
:10693000C0B2E3720C9BE36004F022FF05B0F0BD2F
:10694000F7B50D00019001F033FE071E20D00E2098
:1069500004F0FEFC041E1BD02620FFF731FC061EAF
:1069600000D13E78D0232380C53B0622A370F91DB9
:10697000E01C04F05DFD019B2A0063810123DD40E2
:106980001A401D40210022736573F0B204F0F8FE36
:10699000F7BD0000F0B585B0029010000D001700A3
:1069A0000A9E039301F004FE041E31D0029B002BCB
:1069B0002ED1039B02795B0724D5122313430422B3
:1069C000002E08D10B99002905D10C99002902D17C
:1069D0000D9900291AD01A430D9B2271002B00D06B
:1069E000C9E0002E00D1CFE0002D00D0CCE0606ADD
:1069F000002801D004F094FE1C21300004F090FC2B
:106A0000606205E002239A430E33D7E79343237174
:106A1000654BBA00D458002C00D1AAE0002E10D04B
:106A2000236A002B03D11C2004F0A2FC20625E4BE1
:106A3000BA00D358186A002803D01C22310004F091
:106A4000F7FC0C9B002B12D0574CBB001D596B6AF6
:106A5000002B03D1162004F08BFC6862BB00E358C6
:106A6000586A002803D016220C9904F0E1FC0D9B13
:106A7000002B11D04C4DBC006659B36A002B03D1DA
:106A8000142004F075FCB0622B59986A002803D0DA
:106A900014220D9904F0CCFC380001F089FD051E8C
:106AA00067D0414BBA00D358002B62D01A6A342009
:106AB000002A00D11C389A6A002A01D0143080B212
:106AC0000B9A002A01D01C3080B25B6A002B01D0E7
:106AD000163080B204F03CFC041E4AD0182200217B
:106AE00004F016FE2620FFF76BFB0190002801D171
:106AF0002B780193D0232370029B200063700A231C
:106B0000294EA370039BBD00A371AB59A780196ADE
:106B10001830002905D01C22A06004F089FC200058
:106B200034307359996A002907D0030014221433B2
:106B3000E060029304F07CFC02980B9B002B08D0D1
:106B400003001C221C330B992061029304F070FC9B
:106B500002987359596A002903D01622606104F023
:106B600067FC6B462100187904F00AFE3800FFF735
:106B7000E3FC05B0F0BD10220D9B0D991B69A01818
:106B8000236204F055FC2CE70B9B002B00D13FE760
:106B9000012D00D03CE7606A002801D004F0C0FD60
:106BA0001C210B982AE7C0467064FF1F10B5044CE7
:106BB0002068002803D004F0B3FD0023236010BD3B
:106BC0006464FF1F0B4B07B51A68002A01D100202F
:106BD0000EBD6946531C012012780731FFF772FC85
:106BE0000028F4D002780123100018401A42EED099
:106BF000EEE7C0468064FF1FF0B51F4F01203B68E1
:106C000087B0002B25D09B78059300F0B3FB0028BC
:106C100021D00A20FFF7D4FA04000B20FFF7D0FAA6
:106C2000164B05001E78731E9E413B68F6B2191D77
:106C3000D878FFF757FB3B682900DA7A04330392D0
:106C40009A7901930292009033002000059A04F093
:106C500037FB07B0F0BDFFF7B5FF002805D00620D1
:106C6000FFF7AEFA04000720D8E70820FFF7A8FADC
:106C700004000920D2E7C0466464FF1F6064FF1F60
:106C800070B50A4E040033780D00FF2B0DD00420A0
:106C900004F05EFB011E08D0D0230370CE3B45708C
:106CA0008370C470307804F06BFD70BD0C43FF1F1F
:106CB00070B5040006200D0004F04AFB011E0AD046
:106CC000D0230370CD3B8370054B44701B688580D7
:106CD000187804F055FD002C01D0FFF767FF70BD58
:106CE0006464FF1FF8B5264F06003B680D001124B1
:106CF000002B05D10522234B1B78134202D112240D
:106D00002000F8BD204A10241268002AF8D012781A
:106D1000002AF5D0DB0719D52B789A1E012A1AD83C
:106D20000C2004F025FB132438600028E8D0002351
:106D30000A22437029000670023004F079FBFFF745
:106D40005BFF041E0AD0FFF731FFD9E700F012FB0A
:106D50000028E1D1E4E7002BE2D0D0E70B4B1B7811
:106D6000032BCDD11D20FFF72BFA094B18800028EB
:106D7000C6D0084B04211878074A04F071FCBFE71D
:106D80006464FF1F6164FF1F8064FF1F6064FF1F56
:106D90005E64FF1F8C64FF1F60EA0000F7B501937B
:106DA000194B14001A78052306000F0012201A420E
:106DB00021D0012920D1154B1D68002D1BD00220A8
:106DC0001F2C18D8002C02D0019B002B13D0104B85
:106DD0001F221E706E1C0021300004F099FC0199E6
:106DE0002200300004F024FB310020002C70002F22
:106DF00006D004F00DFDFEBD064B12201D68DCE739
:106E000004F05EFCF7E7C0466164FF1F8064FF1F6B
:106E10000C43FF1F7C64FF1FF8B50F4E122433682C
:106E2000002B17D01B780F3C834213D100250B4F4A
:106E30000221387804F0B4FC094B042138781D8015
:106E400004F0AEFC074B28001D8033685C7004F032
:106E5000FFF904002000F8BD6464FF1F8C64FF1F6D
:106E60007864FF1F5E64FF1F70B5012823D11B4C9F
:106E70002388002B03D01A4A1578002D07D0194B10
:106E80001B68002B02D01878FFF7C6FF70BD3B2BA4
:106E900002D93C3B2380F9E7134E0221307804F0FD
:106EA0007FFCFA222388920002215A43307804F0B2
:106EB0002FFB2580EAE70B4B1B68002BE6D00B4B22
:106EC0001B785B07E2D5084B0221187804F068FCB8
:106ED0000022024B1A80FFF769FED7E77864FF1F94
:106EE0005C64FF1F6464FF1F8C64FF1F6164FF1FED
:106EF000F8B51E4D2868002803D004F011FC0023CB
:106F00002B601B4E3068002803D004F009FC0023DE
:106F10003360184F05243B7818002040234221D0CD
:106F2000154800F02BFA3B78234213D0202004F0C0
:106F30001FFA2860002813D02022002104F0E8FB6B
:106F4000202004F015FA041E306005D02022002114
:106F500004F0DEFB002004E0286804F0E1FB2C6074
:106F60001320F8BD00F00AFAF4E7C0468064FF1F62
:106F70007C64FF1F6164FF1F0043FF1F10B50A4CB4
:106F800023681A1E0ED0002808D10130587004F072
:106F90005FF9002805D02368002B02D00021FFF7FD
:106FA00087FE0122100010BD6464FF1FF7B5274E55
:106FB000050033680191181E21D05C78244F012C04
:106FC00030D1FFF7FFFD002825D02000FFF7F8F8AB
:106FD0000400412814D91F4B022118781E4A04F0DE
:106FE0003FFB1E4B3C3C1C80022233685A703B78AE
:106FF000002B14D128000199FFF75AFE0120FEBD95
:10700000FA2292004243002AEED0124B0221187855
:1070100004F07EFAE8E7FFF7D3F80200F3E7002375
:107020003B70EBE73B78002BE8D1032004F090F9AC
:10703000011E08D0D0230370CC3B457083703368A9
:10704000187804F09DFBFFF7B1FDD7E76464FF1FDC
:107050005C64FF1F8C64FF1F60EA00007864FF1F00
:1070600010B51749838802008B4220D011D81549EA
:107070008B4217D0144900205B1899B2012907D818
:10708000926811785A425341D8B2FFF7F9FD0120B6
:1070900010BD0E4A00209B1807229BB29A42404125
:1070A000C0B2F5E783681878FFF768FFF0E78368F8
:1070B00099785A78090218781143FFF777FFE7E7C4
:1070C0000A20000006200000F8DFFFFFAFDFFFFF0F
:1070D000014B18707047C0460D43FF1F10B5064C9A
:1070E000207001F041FA207804F0F2F905212078AF
:1070F00000F062FD10BDC0468C64FF1F0BB273B57B
:107100000D00002B00DBC4E0884B187804F0B0F9C8
:10711000041E0ED00378912B0FD0A22B00D1A1E03A
:10712000834B1878FF2852D0210004F029FB002857
:107130004DD180200002684076BD43780F2B76D079
:1071400013D8052B70D00E2BEAD18088794B98424A
:107150002BD8794B98421BD8784B9842E0D1A36842
:107160001878591CFFF774F838E03E2BD8D1837893
:10717000032B74D06CD8012B6ED0022BD0D1704B66
:107180001B68002B23D05B68002B20D098471EE0A3
:107190006C4BC0180C28C3D804F062F81DC2C2158D
:1071A0000BC20B0B0B3223C23C00674BC0180728E5
:1071B000B6D8664B1B68002B09D01B68002B06D085
:1071C000200098470AE0A3681878FFF7C7F8200066
:1071D00004F01EF9ADE7A068FFF762F800289FD021
:1071E000F5E7A3681B78002BF1D0554B1B68002BEB
:1071F000EDD01B68002BEAD0210055489847EDE7F9
:107200004F4B1B68002BE2D01B68002BDFD0210006
:107210005048F3E7504B1B68002BD8D05B68002B1D
:10722000D5D021004348E9E7FFF7EAF9CFE78088A6
:107230004A4B984203D04A4B984200D070E7464BE5
:107240001B68002BC3D05B68002BC0D02100D5E7A2
:10725000153B012BBBD963E7FFF798FAB7E7FFF7B8
:107260007DFAB4E73F4B1B78042B07D100236A4615
:1072700013800179408800F0C5FCA8E7364B1B68F5
:10728000002BA4D05B68002BA1D0010036489847A2
:107290009DE7012421420AD0294B1B68002B04D012
:1072A0005B68002B01D000209847012043E78B0743
:1072B0000AD5264B1B68002B04D05B68002B01D03D
:1072C00020009847022036E70421280008400D429C
:1072D00000D131E7254E3388002B21D0013B9BB2F2
:1072E0003380002B1AD1FFF7DBF800280AD0204B9F
:1072F0001C70164B1B68002B04D05B68002B01D060
:1073000020009847FFF7C6F8694601F001FD68467E
:10731000FEF7FEFF1D20FEF753FF308004200AE732
:10732000024B187804F03CFAF8E7C0468C64FF1F63
:107330000D43FF1F0E200000012000000910000077
:107340008464FF1FFEDFFFFFAFDFFFFF8864FF1FC6
:107350000C2000000B2000006C64FF1F0D200000BB
:10736000132000006164FF1FFFFF00005E64FF1F29
:107370005C64FF1F10B501F09BF910BD014B186054
:107380007047C0468864FF1F0B880020162B01D869
:1073900017230420014A13807047C0463664FF1F3C
:1073A00000207047074A03001188814207D0918866
:1073B0000020994202D1013080001018704700204F
:1073C000FAE7C0469464FF1FF0B58F7806000D0001
:1073D000C5B01E2F15D1FFF7E5FF051E03D1002410
:1073E000200045B0F0BD00223B003100C078009283
:1073F00000F0B2FB0400A81C00F0D2FBFF23EB70EE
:10740000EEE7264B062403931B78FF2BE8D0182FBA
:10741000E6D87B08224A013BDB0002929A58944648
:10742000002ADDD0029AD3185B68002BD8D00878E8
:10743000002802D14B78012B02D10624122FCFD184
:1074400007AFAB88697800976446AA68A047041E16
:10745000C6D1AB78029A5B08013BDB00D318390038
:1074600030005B689847041E0BD1AB78042BB6D074
:10747000039A310010782200009700F06DFB0400A1
:10748000AEE76A78002AABD1AA7805A93B880871D3
:1074900030000A704B80FEF747FBA0E71043FF1F48
:1074A00038BA00111D4B37B5050098420BD00029A2
:1074B0000AD1FFF777FF002805D11948FFF772FFBF
:1074C000002800D0058037BD01291AD1FFF76AFFD7
:1074D000041EF8D001235B420380A378FF2BF2D077
:1074E000FE2B07D00023E0781422009329001E33DE
:1074F00000F032FBA01C00F053FB01235B426380D1
:10750000E1E70229DFD1013901F0BEF80028DAD124
:107510002800FFF747FF041EDFD1D4E7FEFF00007D
:10752000FFFF0000022210B5074B52421A800748A5
:1075300001325A809A80DA8000F07EFA044801F025
:1075400025F8002010BDC0469464FF1FC9730011C8
:10755000A57400110388F7B50400002B02D10225A1
:107560002800FEBD42680221137825485268FEF7C4
:10757000A5FD00282ED0234F01253A88002AEFD000
:10758000802321885B0201259B1A9942E8DC0C20AC
:1075900003F0EEFE061E31D03B8822889C46002375
:1075A0001800019561469DB2491989B2AA421BD8BB
:1075B000002801D062443A8000233000082208C02D
:1075C000210003F035FF104A1368002B13D100256A
:1075D0001660C5E76268022113780C485268FEF70E
:1075E0006DFD0028C7D1BAE760681D0140194181CF
:1075F00001330198D6E71A001B68E6E71325AFE7C9
:10760000A6BA00110E43FF1F9064FF1FA4BA001119
:10761000014B18707047C0461043FF1F14230A0027
:1076200010B51A40194204D00122102101F048F887
:1076300010BD4B06F9D4012088434000F8E710B58F
:1076400014008B0604D50122102101F039F810BD79
:1076500008230A001A40194202D14BB2002B0FDA5C
:10766000102101F02DF8002808D02300F2331B78F8
:10767000002BECD0F1342378012BE8D10020E6E791
:1076800003208907FAD4E2E7F0B51F00184B85B054
:107690001C68019002910392002C27D1200005B0B4
:1076A000F0BDA5683301ED186B89019A934211D39F
:1076B000029A93420ED8002F04D10A9B002B10D1BE
:1076C0002C00EBE73B002978039A6868FEF7F6FC8C
:1076D0000028F2D10136B6B2A388B342E1D82468BB
:1076E000DAE7A3680A9A5B891380E9E70026F3E7E3
:1076F0009064FF1F37B50C000A8849880123914226
:1077000017D3002A15D0651D23792A0002210A48C3
:10771000FEF7D4FC102300280BD023796188208841
:1077200000242A000094FFF7AFFF0A23A04200D0F4
:10773000230018003EBDC046A6BA001113B50A00CA
:1077400008884988012388420BD8002809D00024E2
:10775000137905320094FFF797FF0A23A04200D067
:107760002300180016BD13B50A00088849880123B4
:1077700088420BD8002809D00024137905320094E0
:10778000FFF782FF0A23A04200D02300180016BD95
:10779000F0B58BB003904A8808880E00012382421E
:1077A00055D3002853D00023012704AC23700022B6
:1077B000718813000092FFF767FF051E3ED0207806
:1077C000002835D12B78022B18D167706A89830085
:1077D0000130E31880005A8069680222201803F003
:1077E00027FE23780133DBB22370042B19D93B0029
:1077F0006889013080B2002BD9D01FE0022363706A
:10780000122358436A89231804305A806968102269
:10781000201803F00DFE23780133DBB22370002B18
:10782000E5D10C4A6B899B185A425341DBB2DFE722
:107830006378012BE4D12B78022BC7D022780A235E
:10784000002A04D021000398FEF798F900231800BD
:107850000BB0F0BD0100FFFF0F4BF0B5040018683E
:10786000002816D083685D89A54207D88288AE18A3
:10787000B44203DA12019A18934201D10068EFE78B
:107880001E005F891036A74204D1002900D00D8068
:107890001800F0BD3300EFE79064FF1F70B50500DE
:1078A0000C0008880021FFF7D7FF03000120002B00
:1078B00004D022002800197AFFF7C1FE70BDF7B589
:1078C0000C00002501902300EE331B78AB4201D859
:1078D00000200AE06B00E65A00213000E718FFF7AD
:1078E000BBFF002802D126800130FEBD017A01983D
:1078F000FFF794FE002802D03B882380F5E701358E
:10790000EDB2E0E710B5040008880021FFF7A4FFFE
:1079100003000120002B03D02000197AFFF77EFE20
:1079200010BD0000054B1B68002B01D1180004E0BE
:107930009A6852898242F6D1988870479064FF1FF6
:10794000F0B50E27002687B0039302ABFF183E80E8
:1079500005001F4B40891400984207D02B78013056
:1079600000976A6880B2FFF78FFE060002212B782D
:1079700018486A68FEF7A2FB00280FD06C89200027
:10798000FFF7D0FF002802D0013C0419A4B2039BEA
:10799000002B00D01C80300007B0F0BD02212B78F6
:1079A0000D486A68FEF78AFB0028E7D102212B7890
:1079B0000A486A68FEF782FB002807D0002EDED056
:1079C0003B88A342DBD17489013CDFE76C89DEE7A9
:1079D000FFFF0000A6BA0011A4BA0011A2BA00115C
:1079E00010B50C00FFF7DEFC03000220002B0AD0CC
:1079F000002C00D023609B781720FE2B03D0013889
:107A0000FF2B00D1002010BD73B50D0001A90400AB
:107A10001600FFF7E5FF172805D0002E04D1290036
:107A20002000FEF727F976BD01221021200000F08A
:107A300047FE0028F3D0F6E7014B18607047C046B8
:107A4000A064FF1F37B56B469D1D01000400022294
:107A5000280003F0BDFC2B88B02B0ED12379122B0C
:107A600009D12300FA331B78012B06D1012160884C
:107A700000F0E0F801E01B2BF8D037BD10B5054B46
:107A80000421187000F098F8FFF74CFDFEF770FB2A
:107A900010BDC046A464FF1F0020F0B50BB20F005C
:107AA00087B0834234DA274B187803F0E1FC051ED7
:107AB0002BD00378A02B25D103AE3100FEF7E4F8DC
:107AC000041E0BD1B378DB0724D51F4B06341B688B
:107AD000002B03D03100688898470400A86800286C
:107AE00001D003F0D5FD002C08D1184A039B1340A8
:107AF000174A934206D0B3781B2B03D00121688824
:107B000000F098F8280003F083FC80200002784001
:107B100007B0F0BD0F4B1B68002B10D031006888F8
:107B20009847041EDAD07378002BD7D1B27801A918
:107B30000A704B800C716888FDF7F6FFCEE70624CB
:107B4000F1E7C046A464FF1F9C64FF1F00FFFF0015
:107B500000011200A064FF1FF7B50190FC200D008A
:107B600017001E0003F0F4FB04001320002C12D0B9
:107B7000B02320002370089BF42267706580267173
:107B80000830002B08D0190003F052FC21000198A6
:107B900003F0F6FD0020FEBD089903F0B9FDF5E7FE
:107BA00010B5041E06D00078FD2803D803F068FB4A
:107BB000FF23237010BD00000A1F93B210B504000C
:107BC0000220032B05D882400020024BD1529B1883
:107BD0009C7010BDC464FF1F0B8870B5043B04008B
:107BE0000D000220032B0BD80121200000F04CFDDA
:107BF00003001420002B03D02900200000F0DEFB3E
:107C000070BD000007B51300034A00920A0001216D
:107C100000F02CFC0EBDC046417E001107B501925C
:107C200003220092024B0A00122100F049FC0EBD13
:107C3000BF7E001107B56B4601AA11800449D880A8
:107C400008780633012802D1190003F001FE07BDB0
:107C5000A564FF1F0C4B10B518700023FF210B4AC1
:107C60001380138193819380094A5380137051725A
:107C700093819372D174D3821375517703F058FDB9
:107C800000F0FCF910BDC046D464FF1FC464FF1FA0
:107C9000A664FF1FF0B58DB06B46002003910C2247
:107CA0009B5E834200DBB0E05D4B187803F0E0FBA5
:107CB000051E00D1A4E00378902B00D09DE006AF14
:107CC00001004688380000F013FA796804000029A2
:107CD00000D19CE03B88052B6ED13B89032B1CD93E
:107CE00005AC200000F0A2F86288172A61D8398913
:107CF000131D994231D17968237804310291D90753
:107D000038D5607800F08EF9071E06D00023037185
:107D10002378012B08D0132B23D0A868002800D18A
:107D200078E003F0B5FC75E06288029909A800F0DC
:107D3000A6F80290380000F08BF909AA2378387A67
:107D40000192002231000092029A00F012F93800EC
:107D500000F064F9029B002BDFD0300000F080F9C6
:107D6000DBE70378032BD8D16288029909A800F0D9
:107D7000D6F8DEE7122B13D1029909A800F0B5F866
:107D8000021EEAD127498B88002BC6D0887909A921
:107D90002378019161780091310000F0EAF8BCE7A6
:107DA000002302AA93833000617809AAFFF72AFF13
:107DB000B3E71D4B0993F6E7042B02D09A1F012A63
:107DC000ABD8184A043B9B00995A0029A5D0D21879
:107DD000907831003A0000F0AEF800289DD13B8841
:107DE000042B03D001213000FFF724FF012C04D124
:107DF000A868002801D003F04BFC280003F008FB22
:107E00008020039B0002434018000DB0F0BD012804
:107E100000D182E701213000FFF70CFFEDE7C046FB
:107E2000D464FF1FC464FF1F010017000B780370A8
:107E30004B784370CB788A781B021343438070479A
:107E40000A88030002700A88120A42700A88012A0E
:107E500006D14A8882704A88120AC270042070478C
:107E600002208242FBD14A8804309A704A88120A62
:107E7000DA708A881A718A88120A5A71EFE710B587
:107E80000400012082420CD94B780A781B0213436C
:107E90002380834206D1CB788A781B021343638008
:107EA000002010BD022BFBD1CB788A781B02134334
:107EB00063804B790A791B021343A380F0E70B8898
:107EC00003700B881B0A43704B8883704B881B0A16
:107ED000C3708B8803718B881B0A4371CB888371B5
:107EE000CB881B0AC3710820704703000120082AB1
:107EF00014D14A780878120202431A80CA78887826
:107F0000120202435A804A790879120202439A8087
:107F1000CA798879120202430020DA80704710B5CE
:107F200004000120022A05D100204B780A781B02A8
:107F30001343238010BDF8B5060010200F00150074
:107F400003F006FA04000120002C0ED0A0230C221E
:107F5000290023806780201D002D07D003F068FAD8
:107F60002100300003F00CFC0020F8BD03F0D0FB32
:107F7000F6E7F7B51E00009008AB142017001D7837
:107F8000019103F0E5F9041E12D0A2230370019BB6
:107F900047704380099B057146710C220830002B05
:107FA00007D0190003F044FA2100009803F0E8FB21
:107FB000F7BD099903F0ACFBF6E737B5041E0FD007
:107FC0004388002B0CD00025C1881323007A172288
:107FD00001950095FFF7CDFFFF2365806372257043
:107FE00037BD000010B50C4904004A88002A09D0AA
:107FF0008B89002B05D00020CB8A0222834201D03E
:1080000010BD012213000A20434300204032C8540F
:10801000C81842800472F3E7A664FF1F0023438060
:1080200003707047094B00211A0010B55C88002CC2
:1080300006D01C79844203D10A234B43D01810BDCB
:1080400001310A330329F1D10020F8E7A664FF1FAC
:1080500010B50400407A03F013F9FF23637210BDDA
:108060007047043010B580B203F0EAFA002803D05C
:108070000421494203F01CFA10BD000070B5002530
:10808000104CA0682580A581A580A84202D003F0ED
:10809000FFFAA56000250C4C0C4B606D1D80230081
:1080A00058331D70A84202D003F0F2FA656500252E
:1080B0006068002801D003F0EBFA013508340A2D7E
:1080C000F6D170BD6C65FF1F1065FF1F6065FF1F57
:1080D00070B5041E09D1054D2880A881A880A86824
:1080E000002802D003F0D4FAAC6070BD6C65FF1FAD
:1080F000F0B54B8885B00193002343600A790500F1
:108100000F00022A00D07BE0CA88032A17D98B68A7
:108110005E7819783602DC78D8790E4399781B7A24
:1081200024021B020C43034353495BBA0B80331DEB
:1081300093421ED1042C04D0631F022B0ED90120C0
:1081400015E0019A4D4B1201D35A002B06D001982D
:10815000FFF7BEFF4A4A1369013313610421B8686F
:108160002E812C80494203F0A3F96860002005B0FD
:10817000F0BD434D042C06D0631F022B0FD9EB68D2
:108180000133EB60DBE7019A3C4B1201D35A002B21
:1081900005D00198FFF79CFF2B6901332B61374B0A
:1081A00030000293019B029A1B0101930023019965
:1081B0008C468B52130063449C8003939E81FFF78F
:1081C00050FF039B041E986016D00421B8684942F2
:1081D00003F06EF9FA880100043A200003F028F950
:1081E0000199029AFB888A5A043B9B18029A8B5287
:1081F0002B6801332B60A2E7AB690133AB619EE7CB
:108200001E4B0293019B1E01029BF35A002B2DD0A3
:1082100002998C19A068002828D0012A26D1FA8852
:108220009B189BB27352A189994217D39B1AC0180D
:10823000B96803F0FDF8029BA289F35A934200D07B
:108240007DE700222B81A3882B80A3686B60029BB3
:10825000F2520B4A53680133536070E7084A93683F
:10826000013393600198FFF733FF68E7044A5369CD
:1082700001335361F6E7C046D664FF1F6C65FF1FEC
:10828000DC64FF1F70B5051E15D10B4C0B4B18801D
:10829000230058331870606D002802D003F0F8F9FD
:1082A0006565250050356068002801D003F0F0F9BD
:1082B0000834AC42F7D170BD1065FF1F6065FF1F29
:1082C000F0B51700A12285B0920001934243394BCB
:1082D00006001B680C009B18D933FF331D78FDF78F
:1082E00041FF0430854204DD3000FDF73BFF0430E0
:1082F000C5B2BD4207D33A0000213000019B03F014
:10830000BFF805B0F0BD2900380003F041FA2300A2
:10831000C6B250331E700393019B29006365380079
:1083200003F05EF9CBB20293002B02D0039B01361F
:108330001E7000262300503303931B78B34204D8E9
:10834000606D002831D10020DBE7029A2800002A66
:1083500004D0013B1000B34200D02800F700E71919
:10836000387003F075F9786000280ED03A780199DA
:1083700003F05EF8019A3B780136D3180E4A019358
:10838000D369F6B20133D361D4E7039B18706065FB
:10839000A74205D1084A1320D36A0133D362B0E75C
:1083A000606803F075F90834F2E703F071F900230F
:1083B0006365C8E73409FF1FDC64FF1FF7B50D00D4
:1083C00007000421686803F073F82B890400037028
:1083D0002B891B0A43702B8883702B881B0AC37060
:1083E0002E8902250436F6B2F42E15D81B4B9F4277
:1083F00014D10C2002F0ACFF1135011E0CD09023DB
:1084000003708E3B0371043B4380154B8460C68030
:10841000187803F0B5F900252800FEBD5C237B43E6
:10842000104AD3180093583301931B78002B0FD1B7
:108430000300320038000099FFF742FF019B05005E
:108440001B78002BE8D13800009902F071FFE3E7B8
:10845000054A0725536A01335362DDE7FEFF00003A
:10846000D464FF1F1065FF1FDC64FF1FF0B587B0E9
:10847000009017200F0016000193FFF7F2FD13255F
:10848000041E19D00C98031E02D00199201D984794
:10849000030AE370052302AAA070043090812770BC
:1084A0000098667003A993800494FFF787FF051E68
:1084B00002D0200003F0ECF8280007B0F0BD000067
:1084C000F0B587B01F000CAB1B7803910593012119
:1084D0000DAB06001C78049200F0D6F81425002895
:1084E00021D02000FFF77EFD0135041E1BD011496D
:1084F000059B0A7803700132D2B2131EC68001D1E7
:1085000001231A000B7022713000049B039900971D
:10851000FFF7ACFF051E09D1230021000648074ADA
:10852000093303F0D5F8280007B0F0BD00236380BD
:108530002370F8E7D864FF1FBB7F0011307500007F
:10854000F8B505000E00064C064F2368002B02D03C
:108550003100280098470434BC42F6D1F8BDC0462B
:108560007C65FF1F9065FF1F0123064A5B42538015
:10857000002313715362044A136053609360D36005
:10858000136170479065FF1F7C65FF1F0200002389
:1085900010B506499C000859002801D1625010BD51
:1085A0000133052BF6D11320F9E7C0467C65FF1F88
:1085B000034A5388181A43425841404210407047BA
:1085C0009065FF1FF0B585B002930AAB1F780CAB26
:1085D0001B88009008000E0001920393FFF7E8FF4C
:1085E00005001120002D1BD10E48FFF7E1FF04000C
:1085F0001520002C14D006220B99A771E01D02F063
:1086000017FF019B30002371029B29006371009BBF
:1086100066802370039B6562E381FFF791FF28006A
:1086200005B0F0BDFFFF000010B5FFF7C1FF04006B
:108630000220002C12D060880121FFF781FF606AC0
:10864000002801D003F06CF828220021200003F05C
:108650005FF8012300205B426380207110BD0000A1
:1086600030B5074A074C5588010013780020A54211
:1086700004D05B1A59424B415842104030BDC046AD
:108680009065FF1FFFFF0000084A10B501230C0092
:10869000904208D0FFF78CFF031E04D003792340DB
:1086A0005A1E9341DBB2180010BDC046FEFF000009
:1086B000024B1879431E9841C0B270479065FF1F66
:1086C00070B504000D001600FFF772FF002804D1FA
:1086D0000D4B9C4200D0143070BD416A03790520D7
:1086E000002907D012221A40102A02D10520002E9C
:1086F000F2D10F20DB06EFD5897E0C20A9428941FB
:10870000494249420840E7E7FEFF0000030010B578
:10871000002800D110BD0348034A41889142F9D096
:108720009847F7E79065FF1FFFFF0000002330B573
:10873000C45CCD5C6C40D4540133102BF8D130BDF7
:108740000F23002210B5C45C64002243CA54C25CEB
:10875000D209013BF7D210BD0200010010B5203252
:10876000103102F00DFF10BDF0B58BB0039010205A
:1087700005931700049102F0FBFD0090102002F019
:10878000F7FD009B13240190002B05D000280CD18D
:108790001324009802F0C4FF019B002B02D01800A4
:1087A00002F0BEFF20000BB0F0BD102002F0E0FD93
:1087B0000600102002F0DCFD13240500002E00D17D
:1087C000AEE0002819D01022002102F0A1FF3200F3
:1087D0002900039802F0D4FE041E0ED133787F2BBB
:1087E00051D830000099FFF7ABFF009B1B787F2B1F
:1087F00053D801990098FFF7A3FF300002F090FFD3
:10880000002D02D0280002F08BFF002CC1D11020D7
:1088100002F0AEFD0600102002F0AAFD0290002E2C
:108820007CD0002878D03A000F32230001251211A5
:1088300005D00F333B4015B25A4253411BB26A1E5A
:108840001201002B33D0049BD2B298180099029ADF
:10885000FFF76CFF013D10220021300002F058FFAD
:10886000ADB2049F2D017D19AF4242D0002C33D010
:10887000300002F055FF029B002B00D189E7180061
:1088800002F04EFF85E729003000FFF759FF28006E
:108890002549009AFFF74AFFA7E729000098FFF74C
:1088A0004FFF28002049019AFFF740FFA5E70F215D
:1088B0000F4004998A18D9B28F4208D9D15C06A812
:1088C00019540133102BF6D1029A0199C0E7791A95
:1088D00048424141C901F2E73900300006AAFFF7DA
:1088E00025FF3200039806A902F04AFE1037040063
:1088F000BAE7002CBCD13000029906AAFFF716FF98
:10890000320006A9039802F03BFE08220400310061
:10891000059802F08DFDABE71324A9E71324AAE71D
:10892000002800D06EE733E7ACBA0011F0B58BB089
:108930000F0016000225009000283FD0002A3DD0ED
:108940000B1DDBB21800029302F012FD1135041E5C
:1089500034D0FDF747FD05003A000099201D02F0D4
:10896000FFFEEBB20393E3702B0CDBB22F0A0093F4
:108970006370FFB22B0E2370A7700193FDF72CFDDF
:108980001022010006A802F0EBFE2100029A04ABBF
:1089900006A8FFF7E9FE051E0DD1039B08223370E0
:1089A000009B04A9B370019B7770F370301D02F037
:1089B000D7FEFDF71DFD200002F0B2FE28000BB02F
:1089C000F0BDF0B58FB00D00149E03900492059396
:1089D000002A03D1022420000FB0F0BD002EF9D0F0
:1089E0000398FFF7E5FD1424071EF4D0727833785E
:1089F00012021A43B3781B041343F27812061A4387
:108A0000036A0192934201D30133E3D1002D03D0D5
:108A10003B7901249B07DED50822002106A802F03D
:108A200077FE059B13240433DBB21800029302F097
:108A30009FFC051ECFD0059A0499043002F090FEE9
:108A400004223100280002F08BFE39001022103180
:108A50000AA802F085FE2900029A06AB0AA8FFF7D1
:108A600083FE041E0FD1082206A908A802F078FE92
:108A70000822311D08A802F04BFC012807D10199FA
:108A80000398FDF7C9FC280002F04AFEA3E7012481
:108A9000F9E7000070B51C4C05002368181E10D0C3
:108AA000002D14D11A78002A0CD1981C083202F03B
:108AB000BFFC02F015FE0135002808D123681D70A7
:108AC000012070BD0A331800082202F0B1FC2368AF
:108AD000002BF5D0122002F03BFC061E0DD0C12366
:108AE00021680370457002311022023002F0A0FCB0
:108AF00023683100587802F043FE206802F010FE2F
:108B000000232360DCE7C046B865FF1FF8B504000A
:108B10002020FDF755FB0D4EA700BB590500002B8B
:108B20000DD000280BD0D878FF2809D108492A0099
:108B30000C55F35907480333611802F0C9FDF8BD1D
:108B4000290002F0B5FB0028F0D1F8E7D465FF1F3B
:108B5000BC65FF1F659D001170B5064D840063590B
:108B6000002B05D0D87802F08BFBFF226359DA7016
:108B700070BDC046D465FF1F70B506008CB00C00F8
:108B8000150000213022684602F0C2FD310010229B
:108B9000684602F0E5FD1D2021000322684402F032
:108BA000DFFD6846FFF7D8FD2D21040003222800D1
:108BB000694402F0D5FD20000CB070BDF0B507008F
:108BC000160097B001931CAB1D7830221EAB0091AC
:108BD0000AA800211C7802F09BFD102239000AA887
:108BE00002F0BEFD1022002102A802F091FD072232
:108BF000310002A802F0B4FD072202AB9818631EF0
:108C00009C41019902F0ACFD02AB9C732B005A1EF3
:108C1000934102AAD3730021102206A802F078FD26
:108C200006221D9907A802F09BFD1A2002ABC0186E
:108C300006221F9902F094FD102200990EA802F05E
:108C40008FFD102202AB0EA908781C78013A604013
:108C5000D2B2087001330131002AF5D10AA8FFF71A
:108C60007BFD102212A904000EA802F0E1FB1022E5
:108C700006AB0EA908781D78013A6840D2B2087098
:108C800001330131002AF5D10AA8FFF765FD04433D
:108C900010222098E4B212A902F062FD200017B061
:108CA000F0BD70B50E0014008CB0010010226846B3
:108CB0001D0002F055FD3100082204A802F050FD0D
:108CC0002100082206A802F04BFD6846FFF744FD8C
:108CD00004001022280008A902F042FD20000CB078
:108CE00070BDF8B506000D0000243719AC4200D362
:108CF000F8BD02F045FB030A3B70631CDBB2013791
:108D00009D4203D90234F054E4B2EEE71C00EDE7D3
:108D100073B506000C000225002819D0002917D0D1
:108D2000032101A8FFF7DDFF6B469A793F231A4024
:108D3000013313436A463000937101A92200FFF703
:108D40001BFF051E04D10322E01C01A902F070FBE9
:108D5000280076BD03785807DA08C00FD2008000DB
:108D60009B0710439B0F1843C0B2704707230B406B
:108D7000C908C9000B4303707047000070B50400B8
:108D8000FFF7EAFE134DA4006359002B21D0186AA7
:108D9000002801D002F0C4FC2B59986E002801D0A5
:108DA00002F0BEFC2B59D86E002801D002F0B8FCAE
:108DB0002B59186F002801D002F0B2FC2B59586FC4
:108DC000002801D002F0ACFC285902F0A9FC0023D5
:108DD0002B5170BDD465FF1F0E4B8000C35870B57A
:108DE0000C00002B0FD09D68002D0CD02B78201D7F
:108DF0000B706B784B70A97CFFF7B8FF2B7E23724A
:108E00006B69E36070BD10220021200002F080FC3D
:108E1000F8E7C046D465FF1F014B18607047C04695
:108E2000D065FF1F074A03008000825810B5002A52
:108E300006D0D088984203D1012901D1FFF79EFFC7
:108E400010BDC046D465FF1FF0B5264E95B0870013
:108E50000B93BB590500099112200A92002B31D0C7
:108E6000D888FFF7A5FB04001420002C2AD0280086
:108E700010A9FFF7B1FFBB591E781D6A002E23D041
:108E80000895FDF7EFFA07000020FDF7F1FA0790CB
:108E9000A379E61D069310AD0CA9089800F0E2FA3C
:108EA0000EA9280000F0D7FA0B9B0A990493069BA1
:108EB00009980293079B0396019300970EAB0CAAA7
:108EC000FFF77CFE15B0F0BDFDF7CCFA0690300040
:108ED000FDF7CEFAE31DA779079310AB06000893C0
:108EE000DAE7C046D465FF1F30B50C4C85002A591F
:108EF000030085B00120002A0ED018006946FFF754
:108F00006BFF2B591A78D888054B002A00D1054BE6
:108F10006A46072100F0D9FB05B030BDD465FF1FBC
:108F2000579400116594001130B5094C85002959FA
:108F300085B010226846253102F07AFA2A591121AB
:108F4000044BD0886A4600F0C0FB05B030BDC04677
:108F5000D465FF1F0195001130B5094C85002959D2
:108F600085B010226846353102F062FA2A59112183
:108F7000044BD0886A4600F0A8FB05B030BDC0465F
:108F8000D465FF1F3F950011F7B54D4F86001020A7
:108F9000F4590D0002F0ECF9F3592062186A13221B
:108FA00000286CD0033A29009C6802F041FAF3597A
:108FB0001A780192002A58D11E6A227D317B94468C
:108FC00051400122019F114201D167461740217D86
:108FD000914339432175377B4F40BC46604600279B
:108FE000800701D44F081740012102208F40227DC5
:108FF00082433A432275377B5740BC466046002780
:10900000400701D497080F400420227DBF0082430F
:109010003A432275627D002794466046727B424047
:109020000A4201D167460F400121627D8A433A43DB
:109030006275777B5740BC4660460027800701D4A5
:1090400057080F400220627D7F00824317436775F7
:10905000767B00227E40760701D4BA080A400426B7
:10906000617D9200B1430A4362756A78002A08D094
:109070006278002A05D005220533DA770022100035
:10908000FEBD04222979114205D1A17C114202D1F1
:109090000533033AF1E7019A21782C78002A02D1AE
:1090A0000A002100140018220429E8D8042CE6D86C
:1090B00005206043034A05331218525CDDE7C046C1
:1090C000D465FF1FBCBA001110B50A001121024B74
:1090D00000F0FBFA10BDC0469B9500110B0030B5A7
:1090E00087B001AD2B806B4604001100981D08224B
:1090F00002F09EF92A000B212000024B00F0E5FA55
:1091000007B030BDC395001110B50A001121024B04
:1091100000F0DBFA10BDC0461796001113B50B0026
:1091200011006A4613706B4604000622581C02F0B8
:109130007FF96A4608212000014B00F0C6FA13BDF2
:109140003796001110B50A001121024B00F0BDFA4C
:1091500010BDC046879600117FB505000B4BAA00D5
:10916000D4580800002C0FD0666F237FE288217846
:109170000396266F0296E66E0196A46E0094FDF7A4
:1091800009FC2800FFF7FAFD7FBDC046D465FF1F2C
:1091900010B51721FFF7E0FF10BD000070B50A0001
:1091A0000D00064B0221040000F08FFA060029781A
:1091B0002000FFF7D1FF300070BDC0466795001159
:1091C00070B586B000236A461370836804001D786A
:1091D000681E0A2859D801A902F062FA0606333738
:1091E0003B3F43474B4F5300180000F042F9062322
:1091F00012284BD000281BD16088FFF7D9F908232B
:10920000002813D04279002A47D1264B1A78072329
:1092100012070BD5244B1A680723002A06D01668BC
:10922000002E03D0290001AAB04703006A4613703C
:109230006B461B786088002B2AD1FFF767FC06B0CD
:1092400070BD180000F06CF9D4E7180000F087F941
:10925000D0E7180000F093F9CCE7180000F0ADF962
:10926000C8E7180000F0C3F9C4E7180000F0F6F9E9
:10927000C0E7180000F0F6F9BCE7180000F013FA98
:10928000B8E7180000F013FAB4E707236A46137032
:1092900069466088FFF782FFD1E70523012AC5D11F
:1092A000024BB8E76164FF1FCC65FF1FD065FF1F4D
:1092B000F8B52C4F8600F35904000D00002B40D068
:1092C000DA8882423DD15A78062A33D11A78002AA8
:1092D0002ED0012099681A6A097D014206D0157BBB
:1092E000054203D007225A700120F8BD0220014236
:1092F00004D0157B054201D00922F4E70420014285
:1093000004D0127B024201D00B22ECE7164B1B6803
:10931000002BE9D05B68002BE6D020009847BB59B2
:1093200000215B78122BDFD12000FFF715FFDBE770
:109330000E4BECE7112A04D1002900D03225290078
:10934000F2E7002D08D12000FFF732F9002803D002
:10935000102302791343037121002800FDF798FAC6
:10936000C2E7C046D465FF1FCC65FF1FD065FF1F55
:1093700070B50E4E8500AB590400002B13D01B783E
:10938000002B11D10A4B1B68002B04D05B68002B0B
:1093900001D02000984773595B78122B03D100212C
:1093A0002000FFF7D9FE70BD024BECE7D465FF1F2C
:1093B000D065FF1FCC65FF1F094B8000C3581020EC
:1093C000002B0CD01A6A002A09D09B68002B06D00B
:1093D000127A1B7E101C9A4200D9181CC0B270472A
:1093E000D465FF1F70B503000D0014000220002A91
:1093F00030D000292ED013700B78081D53704B7895
:109400009370FFF7A7FCE070012002212B7A2371F3
:109410006B7B034063716A7B0A40134304226371D0
:109420006E7B1640334363716E7BF608F600334360
:1094300063712B7B0340A371287B014000200B4309
:10944000A371297B0A401343A3712A7BD208D2005F
:109450001343A37170BD10B50A0001000120FFF78E
:10946000C1FF10BD10B50A0001000220FFF7BAFFCE
:1094700010BD70B506000C000220002E30D000296F
:109480002ED07378201D0B70B3784B70F178FFF7F6
:109490006DFC01223579257271794B10080013405B
:1094A000934010400343881010408000C9080343D4
:1094B000C9000B436373B1794B100800134093400C
:1094C00010400343881002409200C9081343C900AA
:1094D0000B4321202373FCF773FE854201D2122037
:1094E00070BD2220257AFCF76BFE8542F7D82378E1
:1094F0001820042BF4D86378012BF1D80020EFE773
:10950000030010B50220002909D0002B07D0032248
:10951000481C0A7019000D3201F08AFF002010BDAE
:1095200003000222080010B5002B06D0002904D049
:109530000E32591C01F07CFF0022100010BD030008
:1095400010B50220002909D0002B07D00422481CA6
:109550000A7019000C3201F06BFF002010BD10B52D
:10956000FFF7DEFF10BD03000220002906D0002B0C
:1095700004D0052200200A701B784B70704703004E
:109580000220002B08D0002906D05B7800200B7049
:10959000013B082B00D918307047030010B502209A
:1095A000002909D0002B07D00622481C0A70190098
:1095B0000A3201F03DFF002010BD10B5FFF7B0FFEB
:1095C00010BD02000B00022010B500290ED0002AA9
:1095D0000CD007211970118859701188090A9970E7
:1095E00011180822D81C01F023FF002010BD030031
:1095F0000A00022010B5002B0CD000290AD099785F
:109600005878090201431180901CD91C082201F0EE
:109610000FFF002010BD030010B50220002909D063
:10962000002B07D00822481C0A701900921801F07C
:10963000FFFE002010BD02000B00022010B5002923
:109640000BD0002A09D00921197011781818597007
:10965000511C062201F0ECFE002010BD10B5FFF7F2
:109660005FFF10BD02000B00022010B5002A09D0D8
:10967000002907D05178197011180622581C01F0E2
:10968000D7FE002010BD030010B50220002909D02C
:10969000002B07D00A22481C0A701900063201F07C
:1096A000C7FE002010BD10B5FFF73AFF10BD020045
:1096B0000B00022010B5002A06D0002904D01800A3
:1096C0005178FFF753FB002010BDF0B585B01700AF
:1096D0001E006A4606230500080091819380FEF76C
:1096E000C0FC1324011E02900CD03800B047041EA9
:1096F00005D1280001A9FEF76FFA041E02D00298D6
:1097000001F0C6FF2800FFF701FA200005B0F0BD08
:10971000F0B504008BB0019115000021102202A8C1
:1097200001F0F6FF334EA700B85900283CD0C3889B
:10973000A34239D10378002B36D14278062A18D1BA
:1097400002000100553235310C3006ABFFF7A9FAA3
:10975000002829D12000FFF72FFE020006A902A849
:1097600001F066FE200002A902F06AF801200BB0A9
:10977000F0BD816E002917D00B8A112A28D19D4295
:109780000ED101981231093A01F0C2FD012807D12A
:10979000BB5920009D6EFFF70FFE29000200DEE797
:1097A00032212000FFF7D8FC2000FEF701FF061E43
:1097B0001BD0416A002918D00B8AAB4215D1082270
:1097C0000198123101F0A4FD01280ED1716A0AE05E
:1097D0009D42E9D108220198123101F099FD01283A
:1097E000E2D1BB59996E8A7EB9E7200001F0E0FF13
:1097F000BCE7C046D465FF1FF0B56B4D87007E59AE
:1098000085B0337802900393002B00D087E0B368D3
:10981000346A01937078062817D101221B7D134208
:1098200002D0217B114218D10222134202D0217BA7
:10983000114251D10422134203D0237B134200D0A2
:109840008BE0019B5A7DEB5991E007380428F8D84A
:1098500001F026FF032E42678300B36E002B03D175
:109860001C2001F085FDB066EB599C6E002C1CD0CD
:1098700010220021200001F04BFF0298FFF79CFD11
:1098800001002000FFF72DFA01F07AFD2082200070
:1098900008211230FFF725FA0298FFF78DFDA07618
:1098A000EB592100D888FFF70FFC0822EB591CE088
:1098B000B36E002B05D01A00198AF0881232FFF718
:1098C0000DFC0222019B197DEB5911423DD0207BFA
:1098D00010423AD0073208E0F488FCF7DBFD0100C3
:1098E0002000FFF711FC0A22EB595A70029B9C00E2
:1098F0002A595378073B042B11D8D088FEF758FE1D
:1099000000284ED0C3895A08D2182849029B0298D1
:10991000CB542B5941180433254801F0D9FE05B02A
:10992000F0BDFCF79FFD03000120834201D1002020
:109930000393EB59DE88FCF79BFD0399020030008E
:10994000FFF7ECFB019AEB59117D042211420CD078
:10995000217B114209D00B22C7E7F688FCF73CFDBA
:1099600001003000FFF7EEFB6BE7019A527D012109
:109970000A4204D0607B084201D00C22B5E70221E4
:109980000A4204D0607B084201D00E22ADE70421D8
:109990000A4204D0627B0A4201D01022A5E71222BB
:1099A000A3E7FA225200B0E7D465FF1FD865FF1F76
:1099B0006F9D001110B5064B1A7804231000184053
:1099C0001A4200D00348FFF727FA002010BDC04616
:1099D0006164FF1F1443FF1F70B50400FFF7D4FA42
:1099E000051E43D12000FFF77FFA234EA400A059A3
:1099F0008268937CDB0708D50321036A1B790B403F
:109A0000012B02D1017F0B430377431DD97F8B1EAE
:109A1000022B0DD8022900D00121C088FCF790FF4D
:109A2000042133591A7F59700A431A77280070BDF0
:109A300001290CD102231022437000210C3001F0C7
:109A400067FE305910213530FFF74BF9EEE7052955
:109A5000ECD10223D118437010220C3001F0E8FC45
:109A600004233259117F0B431377EAE7082518289E
:109A7000DCD1053DDAE7C046D465FF1FF0B58BB0F9
:109A8000059143887E4F9E00F45915000493002CE5
:109A900015D1012902D000200BB0F0BD101D577860
:109AA0001678FFF757F9EB68320002932B7A049986
:109AB000019300903B002000FCF70CFFEBE7E388EC
:109AC000049A934201D00820E6E72378012B00D1C5
:109AD000D4E0059B581E092800D9CFE001F0E0FD35
:109AE00005CE0A29CC506C859AB229000498FFF75C
:109AF00073FFD1E7200029001022453001F098FCC7
:109B0000B9594B78042B02D1013B4B70C3E70B00D2
:109B10000A00253335320C310498FFF795F9049883
:109B2000FFF702FA0522431E9841BB59C0005A7044
:109B3000B2E7200029001022553001F079FC049B87
:109B40004F4C9D00295904980A0006AB55320C3140
:109B5000FFF77AF929591022453106A801F0D8FB00
:109B6000012808D10498FFF7F7F90590002804D1DF
:109B700006222B595A7005988EE708230593FAE7B9
:109B800063780C2B7AD1E36E002B03D11C2001F0FB
:109B9000EFFBE066BB59D86E00286FD01022290079
:109BA00001F046FCBB590498DC6EFFF705FC0D2262
:109BB000A076BB595A706EE7E06E00285ED06378DD
:109BC0000D2B5BD12B8808220382A91C123001F0D7
:109BD0002FFCBB599A68517D0222114226D0186A87
:109BE000407B104222D00C32E4E763780E2B45D143
:109BF000236F002B03D1162001F0BAFB2067BB595D
:109C0000186F002803D01022290001F011FC0F2248
:109C1000BB59CFE763780F2B30D1206F0622691C28
:109C2000103001F005FCBB599A68517D04221142A5
:109C300003D0196A497B1142D5D100210498FFF75E
:109C40008BFA28E7636F002B0DD0BB59586F0028A3
:109C5000F3D01022290001F0EBFB0122BB59524244
:109C60005B6F1A61E9E7142001F082FBBB59606762
:109C70005B6F002BE9D126E72978DFE707200BE7A8
:109C8000D465FF1F10B5064C207001F0C1FC062101
:109C90002078FDF791FF0348FEF778FC10BDC04621
:109CA000E765FF1F258E001100200BB270B50D0077
:109CB000834216DA264B187801F0DAFB041E0DD029
:109CC0000378922B0ED0A02B37D0224B1878FF2888
:109CD0003AD0210001F054FD002835D18020000247
:109CE000684070BD43780E2B0BD03E2BEDD18378AE
:109CF000052B12D0082BE8D181798088FFF7D8FA9C
:109D000008E0154B82889A42DFD183681878591C85
:109D1000FEF7C0FE002817D1D7E7104B1B785B0772
:109D200012D50F4B1B68002B0ED09B68002B0BD05D
:109D3000C289811D80889847ECE7FFF741FAA06847
:109D4000002801D001F0A4FC200001F061FBC5E770
:109D5000E765FF1F0D43FF1F182000006164FF1F10
:109D6000D065FF1F10B50078FFF712FA10BD10B5CF
:109D70000078FFF7FDFA10BD0C234343084A10B5E5
:109D80009B185A68002A03D0012901D1904710BDC1
:109D90009B68002BFBD00029F9D19847F7E7C04614
:109DA0000466FF1F01238340094A10B5946B1C43CE
:109DB0009463506B98435063D46B200098430129FF
:109DC00001D120001843D063116B0B43136310BD06
:109DD00000800040F0B500240127154B85B0DA6BF8
:109DE000144E03921A6C0192DA64019BE3403B42E9
:109DF00017D0039DE5403D400295E5B20299280049
:109E0000FFF7BAFF316A736A002908D03900002BC6
:109E100001D0029979402800FFF7C4FF01E0002B30
:109E2000F9D101340C36172CDFD105B0F0BDC04696
:109E300000800040E865FF1F064B01215A68C240C0
:109E40000A4204D01B68C3401800084070471B6DCD
:109E5000F9E7C046008000400122064B82400029FD
:109E600003D0D9680A43DA607047D9689143D96052
:109E7000FAE7C0460038004030B5032444430F4B96
:109E8000E25C1B199C785D7801232D1B0135AB40EA
:109E9000013BA340A140DB430C00122807D808492E
:109EA00092005218116819402143116030BD054AD3
:109EB00011680B4023431360F8E7C04603BB001151
:109EC00008F0004014F00040C21F70B5D4B2062361
:109ED000092C0BD80125084C9540002908D00021F9
:109EE000FFF7CAFF23682B4323600023180070BDCF
:109EF0002368AB43F8E7C04600380040214BF0B57B
:109F00001B185B78022B21D1032444431E4A1F4EA9
:109F1000A35C12199478012215008540B76B013CAF
:109F2000E4B23D43A240B563194C122815D89B00FA
:109F300000290CD117495B1899680A439A600123DC
:109F4000205C154A834011680B431360F0BD114932
:109F50005B18996891439960F1E70E4B00290DD188
:109F600059690A435A61225C1328E8D00123203A38
:109F700093400A49086803430B60E7E75969914336
:109F80005961F0E7E865FF1F03BB00110080004046
:109F900048BB001100F00040A0F00040A4F00040D9
:109FA000F8B500241B4E1C4D1C4B1B5D012B1FD113
:109FB000194A9269E2401A420BD00122B2569340EC
:109FC0002200143AD2B2022A09D815494A69134329
:109FD0004B61013402360C35172CE5D1F8BD002257
:109FE000B2560F499200521891680B439360F0E704
:109FF000022BEED1E7B23800FFF71EFF01235840D5
:10A00000C1B23800FFF77AFF3800FFF715FF687715
:10A01000DFE7C046D5BA0011E865FF1FE965FF1FFD
:10A0200000F00040012202388240054B002903D095
:10A0300059690A435A617047596991435961FAE76E
:10A0400000380040F8B50E0001210F008740114A8A
:10A050000400D368FD43BB43D360831E8B4201D809
:10A06000FFF7E0FF00212000FFF72EFF0A4A0B4B0D
:10A070005168012E05D139431B1951605E700020D3
:10A08000F8BD2940516002221C1962709A6915407E
:10A090009D61F4E70038004000800040E865FF1F44
:10A0A000012210B58240074B002906D019680A43E7
:10A0B0001A600121FFF7C6FF10BD196891431960AE
:10A0C000F7E7C046008000400C2370B500254343ED
:10A0D0000A4A29009B181D70094B04001B185D706B
:10A0E000FFF7B0FF0123A340064928000A681A437E
:10A0F0000A6005490A689A430A6070BD0466FF1F3A
:10A10000E865FF1F348000403080004070B50400D7
:10A110000E00FF2813D003250540FFF7D5FF084A9E
:10A12000A3089B009B183F22ED00AA40AE4019688F
:10A1300020009143314319600121FFF78DFE70BD6E
:10A1400018380040F8B50C244443134B0500E418BC
:10A150006368002B03D1A3681220002B1AD00222BF
:10A1600001270E4B00215B195A7028002770FFF75A
:10A1700069FF63681E1E08D0A3683E00002B04D050
:10A180002800FFF759FE4640F6B228003100FFF7DD
:10A1900009FE0020F8BDC0460466FF1FE865FF1FEA
:10A1A000F7B5C420FF222B4B80001958002491439F
:10A1B0003F3A0A431A508022274F5202274E1A6014
:10A1C000274B1D5D002D21D0A31E012B03D801219B
:10A1D000E0B2FFF727FF012D18D11F4B9B69E34029
:10A1E0002B4213D0E3B218000193FFF725FE0100C4
:10A1F0000198FFF755FFE3B2143B022B1DD8012154
:10A200007156184A8D405369AB4353613B7F002B15
:10A210000DD0E5B22800FFF795FF2800FFF70CFEF0
:10A220007B7F0100834202D02800FFF7A5FD0134A7
:10A230000C370236172CC3D1F7BD0121002371560C
:10A24000F3568D40074A9B009B189A68AA439A6070
:10A25000DCE7C04600E100E0E865FF1FD5BA001169
:10A26000E965FF1F00F0004010B501210400FFF771
:10A27000E9FE0123044A002011194B70A3409169A3
:10A280000B43936110BDC046E865FF1F70B50E001B
:10A2900015000400FFF718FF0C236343094A200050
:10A2A0009B189D605E60FFF74DFFF021064B074A4B
:10A2B0008900051E5A5002D02000FFF705FF280034
:10A2C00070BDC0460466FF1F0000FF1FD59D001132
:10A2D00070B5134D07202C78002C1FD19822210037
:10A2E0005200280001F06CFA0123C420FF222B70D9
:10A2F0000C4B80001C635C630B4B1C605C600B4B65
:10A30000195891433F3A0A431A50802252021A6068
:10A310000D20074A074900F0BBFF200070BDC04672
:10A32000E865FF1F00800040A0F0004000E100E071
:10A33000A1A10011A19F0011030010B50620072B59
:10A3400009D8054A137001F043FAD7210020034BC6
:10A35000034A89005A5010BD3C43FF1F0000FF1FF5
:10A360008D1BFF1F70B51D0002240C2910D8094A4F
:10A37000CA40D2070CD5FBF72FFF041E08D1059A5F
:10A3800004992800FBF744FFFCF7B2FDFFF712FB2E
:10A39000200070BD1210000030B50D7802232C0093
:10A3A0009C43184201D02B431C0008252300AB43DB
:10A3B000284201D02B00234320241D00A543204226
:10A3C00001D01C4325002A230D70184204D01178B7
:10A3D0001E3B0B43137030BD0028FCD10C211378B9
:10A3E0008B43F7E7F8B51D0006AB1B88140007AADE
:10A3F0000E000B201778002B27D10A78022A49D1AA
:10A400004A68507811780002244A084380180428CA
:10A4100040D801F045F903121D1B2300F06801F03C
:10A4200007FA021CC0B2B84200D93A1CD2B22000CE
:10A43000F1682A8000F0FCFF06E00222F3681B8826
:10A440002A8023701B0A63700020F8BD0622EEE705
:10A4500001232B80F3681B782370F5E7F368002B4A
:10A4600016D008222A801A8822701A88120A62706E
:10A470005A88A2705A88120AE2709A8822719A88C1
:10A48000120A6271DA88A271DB881B0AE371DBE7CA
:10A490002B80D9E701202B80D7E7C04600D6FFFFED
:10A4A000F7B516000A781D0008AB1F880C000123C1
:10A4B000022A18D14A685078117800022B4A0843C2
:10A4C000801803280FD801F0EBF802254439E06822
:10A4D00001F0AEF9C0B20723B84204D37B1901934F
:10A4E000152B02DD0D231800FEBDE0682A003100A7
:10A4F000C01900F09DFF6B4600209B88E268D05495
:10A500001B4B1B68834203D01B68834200D09847D3
:10A510000023E8E70B23002FE5D1022DE2D1737869
:10A5200032781B021343E2681380114B1B68002B27
:10A53000EED01B68002BEBD00120E8E70B23002FA7
:10A54000D1D1062DCED12A003100E06800F070FF95
:10A55000DEE70B23002FC6D1012DC3D1327875332E
:10A56000012AC0D8E3681A70D2E7C04600D6FFFFC0
:10A57000F467FF1F70B50C001500072837D801F0ED
:10A580008FF8041436361B36242E182015290BD8C4
:10A59000184E16220021300001F0BAF822002900DE
:10A5A000300000F045FF002070BD18200229FBD1CB
:10A5B0001288114B1A80F6E718200829F4D10A00F6
:10A5C0000E48290000F004FFEDE718200129EBD127
:10A5D0000B4B10780B49DA69FFF7DEFEE3E7182032
:10A5E0000129E1D1064B10780749DA6BF4E7022024
:10A5F000DAE7C046DC67FF1FBA43FF1FB043FF1F07
:10A600004043FF1F6843FF1F8843FF1F030010B52F
:10A610000020DB0704D50721024A034800F08CF82C
:10A6200010BDC04660BB00114043FF1F054A030038
:10A630001068002803D082889A4201D18068704750
:10A640000068F6E7EC69FF1F0A88030008009A42D9
:10A6500004D08A8804309A4200D00020704700005D
:10A66000F8B5F22200230D4F0D4E796805004243E4
:10A670003370994200D07B600A4C0021200001F029
:10A6800047F800231A007C60AB4202D100203370EF
:10A69000F8BD01332280DBB2F234F5E7E46AFF1F34
:10A6A000E26AFF1FF069FF1F73B56B460190060059
:10A6B000684615001980FCF74DFF041E11D1002DCE
:10A6C0000FD07689002E11D00C2000F051FE00280A
:10A6D0000ED0084A0460136886808560002B02D182
:10A6E0001060200076BD1A001B68F7E70224F8E727
:10A6F0001324F6E7EC69FF1F012100220A4B10B575
:10A7000049420A4C198099809A719A70084B2070BE
:10A71000012019805A60FFF7A3FF2078FCF778FF2B
:10A720000448FDF733FF10BDFC67FF1FEC6AFF1FF5
:10A73000E46AFF1FE5A70011022310B5002802D02C
:10A74000FFF7B2FF0300180010BD0000030010B5B2
:10A750000020DB0704D50421024A0348FFF7A4FFC9
:10A7600010BDC04674BB0011C043FF1FF0B50E26DC
:10A7700087B003930CAB1F8802ABF61805000800E6
:10A7800031000292FDF768F804000120002C0FD080
:10A790003088FFF74BFF03000E20002B08D05E68C7
:10A7A000002E05D021002800039B029A0097B04795
:10A7B00007B0F0BD0A4B10B5984207D10122002323
:10A7C00052420A808B708A808B7110BDFFF73CFF6C
:10A7D0000028FAD001235B42038000238370F4E752
:10A7E000FFFF0000F8B5050001290AD1134E00242F
:10A7F0003388F227AB4219D028001149FFF7DAFF5E
:10A8000006E0022904D10139FDF73EFF0028EDD012
:10A81000F8BD3B0063437268D018D35A002B09D0AF
:10A820003A00002100F074FF0134E4B2054B1B78BC
:10A83000A342EED801235B423380DDE7E46AFF1FC9
:10A84000FC67FF1FE26AFF1F10B5FFF7FDFE030064
:10A850000020834200D0987810BD0000F0B589B088
:10A860001C000EAB80CB03901E8810AB1B780492AB
:10A8700002930B7A0D00DB0616D42B780593022B7E
:10A8800024D00498FFF7D2FE002812D003689C461B
:10A89000002B0ED0029B2200019329003B0064464E
:10A8A00003980096A04705E00498FFF7BFFE002834
:10A8B00002D10E2009B0F0BD8368002BF9D00A2226
:10A8C0002900039898470028D7D0F3E76B68587899
:10A8D0001A786B4B000210439842D2D8043B98423E
:10A8E00010D2684B984242D015D8674BC018012847
:10A8F000C7D80B20002EDDD1EB681A7859683A8052
:10A90000200028E0614BC018032800D979E000F04E
:10A91000C7FE846A789E5E4B9842B2D10B20002E0F
:10A92000C8D101233B80EB6831001B782370688914
:10A93000013080B2FCF790FF3A88031E0ED00178F8
:10A9400002328A183A80428962704289120AA270E1
:10A9500059680278E01C00F06BFD06E004323A8092
:10A9600031000422601C00F0D3FE0020A2E70B207F
:10A97000002E9FD1EB6807A91E8804233B80330A71
:10A98000300026706370FCF767FF051E28D004AB0B
:10A990009A890E2304A95B183E49C668FCF7D0FFCC
:10A9A00000280BD12B783C486A680599FBF786FB99
:10A9B000002803D1012304AA5B42D3813278022A02
:10A9C00006D17168201D00F033FD3B8802333B80C7
:10A9D0000E2304AA9B181B88A3701B0AE370C4E70C
:10A9E00004ABDE81F4E70B20002E00D062E7E968BB
:10A9F0000398FFF729FF02233B802070000A607054
:10AA0000B3E70B20002E00D054E70222EB681B882E
:10AA10003A8023701B0A6370A7E7E86800F008FF1C
:10AA2000C2B203000720B24200D243E70DD0029920
:10AA3000DBB27118994202DB921BD3B20293029BE4
:10AA4000E9681A003B8089195AE70023F6E70B20D2
:10AA5000002E00D02EE70722EB683A801A78227089
:10AA60005A7862705A88A2705A88120AE2701A796B
:10AA70002271DA886271DB881B0AA37175E7C04610
:10AA8000042900000228000000D8FFFFFFD6FFFFC6
:10AA900003280000FFFF0000A4BA0011F0B58DB03C
:10AAA0006B460020089120229B5E83423DDAA64B34
:10AAB000187800F0DDFC071E32D00378B02B2CD1C3
:10AAC0000079023816281FD800F01AFC17001E0063
:10AAD0001E001E0031001E0096001E001D011E00FB
:10AAE00052011E0073011E00CD011E0050021E0007
:10AAF0001E001E008E021E00E302944B94491B8828
:10AB000078880B80FBF71AF83800FCF79BFF914B15
:10AB10001B68002B01D038009847380000F078FC03
:10AB20008020089B0002434018000DB0F0BDEE22CB
:10AB30000021874800F0ECFD0BAA3B7B798938891E
:10AB400000923A000D32FCF79FFD0400804B1B7809
:10AB5000002C3FD146E0804B788805937F4B410025
:10AB6000CB5A0BAE073BDBB2328802930023019332
:10AB70007B4B210006930093059BFFF76FFE744DFE
:10AB8000002810D1069B3A8A1B889A420BD13800C4
:10AB90000599123000F0BCFB002804D02B786289A4
:10ABA0009B00EB185A80162306A81B183288200039
:10ABB0007989FCF7C5FE2B7804009A00AA18518801
:10ABC0000029C3D00133DBB22B70002807D006A9BF
:10ABD000C98A9180634A12889A42BCD802E0012156
:10ABE00049429180002B04D059497888FAF7DAFF5E
:10ABF0008AE73E890A2479E000253E89574B06936F
:10AC00007B88069A5B009B5A033B9D4202DB002D2A
:10AC1000F0D05BE0162206A812183B7B79890092DF
:10AC20003A0030000D32FCF72FFD0590002858D077
:10AC30004689017A7888FCF7F1FC041E44D1464B22
:10AC400078880793069B4100C95A454B0439C9B21D
:10AC500006AAD28A06930291019400930599079B54
:10AC6000FFF7FCFD041E2FD1069B39491A88931C5F
:10AC7000002D26D14B807988384B4900CB5A511989
:10AC8000033B8B4220DD059B31485B8941190B71E9
:10AC9000A91C0135C9B2EDB2059145191B0A2B71EA
:10ACA000059B2D490433181800F0C2FB2C4B059A64
:10ACB0001B88D318DDB22C4B9E4205D00136B6B2AC
:10ACC0009CE749889942D6D0002D0CD0204C280012
:10ACD000618800F035FD207021007888FAF772FF56
:10ACE00012E7059CF0E7002C00D183E77B78142B5A
:10ACF00000D109E716493B794E800B700C717888BA
:10AD0000FAF712FF00E7162406ABE4182100388991
:10AD1000FCF7A2FD011E00D1B7E1788822880F4C14
:10AD200045002C5B0A4D013CE4B2029400240F4B19
:10AD300001940095FFF792FD041E00D014E1290054
:10AD40007888FAF74FFFDFE6EC6AFF1FAC42FF1F7F
:10AD50000468FF1FF867FF1FF868FF1F3464FF1FB8
:10AD6000E869FF1FAA42FF1FFFFF00000668FF1FE0
:10AD7000162406ABE41821003889FCF76DFD011E8E
:10AD800000D182E178882288AE4C45002C5BAE4D24
:10AD9000013CE4B202947C89AC4B01940095FFF72E
:10ADA0005DFD041E00D0DFE029007888FAF724FF5B
:10ADB000AAE60025A44B1D803B00F6331B78A24A6F
:10ADC00078880792AB4208D99E4B12880693069961
:10ADD00043005B5A013B9A4203DB0799FAF716FFDF
:10ADE00092E616246B00FB18059306ABE418059B4E
:10ADF00021001889FCF730FD011E03D1059B0124B9
:10AE00001E8973E77888924B2288069C0993430039
:10AE10001B5B904E013BDBB2029300230096019333
:10AE2000099BFFF71BFD041E02D0059B1E895DE7F1
:10AE30007B88069A5B009B5A079A10883288121802
:10AE4000934202DC1B1A013B33807F4C0230328874
:10AE50000999001900F0ECFA2388328801359B1813
:10AE60002380EDB2A8E70BAA3B7B79893889009251
:10AE70003A000D32FCF708FC00250590059B002BDD
:10AE800004D10A24002D00D16EE060E0059B788893
:10AE9000197AFCF7C3FB0100041E63D1694C6C4BAB
:10AEA000788806940993069B4400E45A694B063C53
:10AEB000E4B20BAE32880793029401910093059996
:10AEC000099BFFF7CBFC041E4CD1079B5E491B88F6
:10AED0001A1D002D30D14A80059B5B4C5A8963199D
:10AEE0001A716B1C9BB2E318120A1A71162306A87A
:10AEF00032881B1879890598FCF722FDFF21AA1CCE
:10AF00002E1D03350B00059092B2B6B2ADB20028EB
:10AF100003D006ABDB8AD9B21B0AA21865191171DE
:10AF20002B714C4D301D2A884949201800F080FAB9
:10AF30002B88F618B5B2A1E74988914207D17A88E3
:10AF400006995200525AEB18053A9A42C4DC3E4C1C
:10AF50002800618800F01CFC207021007888FAF736
:10AF60005FFED1E5002DF2D13E89BFE6162606AB85
:10AF7000F61831003889FCF76FFC3D000400FA3503
:10AF800000282DD0037A9B060CD400227B893989B6
:10AF9000788800923A000C32FFF7E8FB041E10D0CC
:10AFA0003E8915E03088FFF741FB00281AD08368FE
:10AFB000002B17D02100122278889847041EE4D075
:10AFC000EEE72B78002B02D17888FAF739FE0026BD
:10AFD0002B78002B00D097E5002C00D194E585E676
:10AFE0000124DDE70E24DBE7162506ABED1829006A
:10AFF0003889FCF731FC041E47D0037A9B0611D434
:10B00000154A7B881188994203D01448814207D1A0
:10B010001380134BF2261D780023D9B2A94221D305
:10B020000924A1E72888FFF701FB00282FD08368B7
:10B03000002B2CD02100122278889847041EDFD0E4
:10B0400092E7C0463464FF1F0468FF1F0668FF1FB5
:10B05000F868FF1FE869FF1FE46AFF1FFFFF000099
:10B06000E26AFF1F31005943546801336018615A86
:10B070000029D2D13C0008342100F22200F0D8F996
:10B0800021007888FAF7E4FD3EE501246CE70E2400
:10B090006AE71D4B1A887B889A4231D07888FAF784
:10B0A000E1FD31E5F223059851684343CD18C95AB3
:10B0B00000291FD03B7A012B0BD16C88AB88788894
:10B0C000AA1D0094FFF752FB041E02D000233B721E
:10B0D0002E88F2220021280000F01AFB00232B808A
:10B0E000059B0133DBB20593084B05991B78064A93
:10B0F0008B42D7D801235B421380002CCED0F5E5DC
:10B10000002634000596EFE7E46AFF1FE26AFF1F9E
:10B1100070B504000E001500FFF796FA031E08D163
:10B1200031000548FFF790FA03001120002B02D0F0
:10B130001C8000209D7070BDFFFF0000F8B50B4F14
:10B1400006003B780D001400FF2B0ED00A2000F003
:10B15000FFF8011E09D0B12303800023468003714C
:10B16000C5800481387800F00BFBF8BD0144FF1F57
:10B17000F7B50F0008A90600088809A90B2409885B
:10B18000002821D10234022B1ED1557813782D02CC
:10B190001D432B008B4301937334002B14D1FB68A8
:10B1A000300019000093FFF74FFB019C85420BD044
:10B1B0002A0030000099FFF7ABFF041E04D12A00DB
:10B1C00030007989FFF7BAFF2000FEBDF0B50E7898
:10B1D00085B003900AA805880120022E0DD14C6885
:10B1E0002778647824023C43054FBC4205D103987C
:10B1F000DBB201960095FFF7BBFF05B0F0BDC0467E
:10B2000002290000034B10B51B68002B00D09847A3
:10B21000FEE7C046F06AFF1F07B501A8FFF7F2FF7F
:10B22000044A05480021121A00F0CAFAF8F7EAFAAF
:10B23000FEE7C046F46AFF1F0444FF1F0000000041
:10B2400001B40248844601BC604700BF3D36FF1F81
:10B2500001B40248844601BC604700BF691F00007A
:10B2600001B40248844601BC604700BF093BFF1F90
:10B2700001B40248844601BC604700BFF30E0000E1
:10B2800001B40248844601BC604700BF1147010079
:10B2900001B40248844601BC604700BF0D31FF1F66
:10B2A00001B40248844601BC604700BF214601004A
:10B2B00001B40248844601BC604700BF5147010009
:10B2C00001B40248844601BC604700BF851F0000EE
:10B2D00001B40248844601BC604700BFF137FF1F3C
:10B2E00001B40248844601BC604700BF1D4B010009
:10B2F00001B40248844601BC604700BFDD6601001E
:10B3000001B40248844601BC604700BF313BFF1FC7
:10B3100001B40248844601BC604700BFCD4C010027
:10B3200001B40248844601BC604700BFF94C0100EB
:10B3300001B40248844601BC604700BF3119FF1FB9
:10B3400001B40248844601BC604700BFA54F01001C
:10B3500001B40248844601BC604700BF1D4D010096
:10B3600001B40248844601BC604700BF3D37FF1F5F
:10B3700001B40248844601BC604700BF3D4B010058
:10B3800001B40248844601BC604700BF2951010056
:10B3900001B40248844601BC604700BF9DA900007B
:10B3A00001B40248844601BC604700BFB14E0000B2
:10B3B00001B40248844601BC604700BF3139FF1F19
:10B3C00001B40248844601BC604700BFC53AFF1F74
:10B3D00001B40248844601BC604700BF810E0000F2
:10B3E00001B40248844601BC604700BF156B0100F0
:10B3F00001B40248844601BC604700BF8552010089
:10B4000001B40248844601BC604700BF7139FF1F88
:10B4100001B40248844601BC604700BF434D0100AF
:10B4200001B40248844601BC604700BF012400000B
:10B4300001B40248844601BC604700BFE94C0100EA
:10B4400001B40248844601BC604700BF3D180000BB
:10B4500001B40248844601BC604700BFED3AFF1FBB
:10B4600001B40248844601BC604700BFE538FF1FB5
:10B4700001B40248844601BC604700BFF54E01009C
:10B4800001B40248844601BC604700BF0519FF1F94
:10B4900001B40248844601BC604700BF75A90000A2
:10B4A00001B40248844601BC604700BFADAE000055
:10B4B00001B40248844601BC604700BF5549010001
:10B4C00001B40248844601BC604700BF212400004B
:10B4D00001B40248844601BC604700BF5D1700000C
:10B4E00001B40248844601BC604700BFC51D00008E
:10B4F00001B40248844601BC604700BF6D30FF1FA5
:10B5000001B40248844601BC604700BF056A0000E0
:10B5100001B40248844601BC604700BF8B52010061
:10B5200001B40248844601BC604700BFED4A0100F7
:10B5300001B40248844601BC604700BFAD32FF1F22
:10B5400001B40248844601BC604700BF455000007A
:10B5500001B40248844601BC604700BF5125000089
:10B5600001B40248844601BC604700BFEDA500005D
:10B5700001B40248844601BC604700BFF938FF1F90
:10B5800001B40248844601BC604700BFE5480000A2
:10B5900001B40248844601BC604700BF3555000035
:10B5A00001B40248844601BC604700BFB54C0100AD
:10B5B00001B40248844601BC604700BFC5210000B9
:10B5C00001B40248844601BC604700BFC56D01005C
:10B5D00001B40248844601BC604700BF8530FF1FAC
:10B5E00001B40248844601BC604700BF090E000058
:10B5F00001B40248844601BC604700BF993AFF1F6E
:10B6000001B40248844601BC604700BF0D520100EE
:10B6100001B40248844601BC604700BFC92600004F
:10B6200001B40248844601BC604700BFC9A90000BC
:10B6300001B40248844601BC604700BF055E0000BB
:10B6400001B40248844601BC604700BFE9280000FD
:10B6500001B40248844601BC604700BF017F00007E
:10B6600001B40248844601BC604700BF5952010042
:10B6700001B40248844601BC604700BFC94A0100CA
:10B6800001B40248844601BC604700BF6D36FF1F0D
:10B6900001B40248844601BC604700BFD94901009B
:10B6A00001B40248844601BC604700BF1D3BFF1F38
:10B6B00001B40248844601BC604700BF4936FF1F01
:10B6C00001B40248844601BC604700BF5522000017
:10B6D00001B40248844601BC604700BFA94601008E
:10B6E00001B40248844601BC604700BFD91B00007A
:10B6F00001B40248844601BC604700BF0534FF1F07
:10B7000001B40248844601BC604700BF456B01009C
:10B7100001B40248844601BC604700BF154D0100DA
:10B7200001B40248844601BC604700BF014C0100DF
:10B7300001B40248844601BC604700BF791800008C
:10B7400001B40248844601BC604700BF350E0000CA
:10B7500001B40248844601BC604700BF2D2EFF1F84
:10B7600001B40248844601BC604700BF4551010056
:10B7700001B40248844601BC604700BFB139FF1FD5
:10B7800001B40248844601BC604700BF594F010024
:10B7900001B40248844601BC604700BF090E0000A6
:10B7A00001B40248844601BC604700BFB3520100A7
:10B7B00001B40248844601BC604700BF091B000079
:10B7C00001B40248844601BC604700BFB70E0000C8
:10B7D00001B40248844601BC604700BF8D1BFF1FB7
:10B7E00001B40248844601BC604700BF291C000028
:10B7F00001B40248844601BC604700BF6DBC000034
:10B8000001B40248844601BC604700BF6571010075
:10B8100001B40248844601BC604700BF4D1F0000D0
:10B8200001B40248844601BC604700BF25260000E1
:10B8300001B40248844601BC604700BFDD520100EC
:10B8400001B40248844601BC604700BF311B0000C0
:10B8500001B40248844601BC604700BFE117000004
:10B8600001B40248844601BC604700BF1D3AFF1F77
:10B8700001B40248844601BC604700BFD532FF1FB7
:10B8800001B40248844601BC604700BF8D1200002D
:10B890000001010302030303040305020602070279
:10B8A000080209000A030B030C020D000E030F032C
:10B8B000100311031303140315001600C53B0011F8
:10B8C000F93B00110000000002000000D2B8001196
:10B8D000192A0F180A000000F1590000FD24000089
:10B8E00041460100957C0011A99C0011FD700011DA
:10B8F000997A0011A95200119DAA0011FD4E001164
:10B90000D53D0011053F0011000000001616000093
:10B91000020000001CB90011F4FFF3FFD2FC00008C
:10B9200045400011000000000000000054757961DE
:10B930000042312E39003030313400676974687547
:10B94000622E636F6D2F70767678004254483031E6
:10B95000000000000200000068B90011292A282A0E
:10B96000272A262A252A242A0A180000E204000091
:10B970007102000078EC0000050000007440000037
:10B980001027000060F000000400000006640000C2
:10B99000204E00000000000006000000050000002E
:10B9A0001F501D00023CB4000001140019000000EB
:10B9B0008102000030313233343536373839414274
:10B9C0004344454600000000AD56001101570011E8
:10B9D0000000000002000000E0B900116F2A6E2A8A
:10B9E0001A18000001A00000000000006410B71D3C
:10B9F000C8206E3BAC30D9269041DC76F4516B6B9D
:10BA00005861B24D3C7105502083B8ED44930FF05E
:10BA1000E8A3D6D68CB361CBB0C2649BD4D2D38614
:10BA200078E20AA01CF2BDBDFB349B5F8000008061
:10BA30000010000000000000FF5C0011897300117D
:10BA4000235D001191770011A75D00116777001148
:10BA50001D5E00113D7700116F5E00110579001128
:10BA6000D75E001105790011095F0011BF78001140
:10BA70001D5E0011F5760011955E00119D78001194
:10BA800000000000000000007B5F00119D780011A5
:10BA9000DD5F0011A1730011052A042A012A002A82
:10BAA00002290328012800280118001800000000BE
:10BAB00000000000000000000000008701010201FA
:10BAC000020101020102030304010301010101015A
:10BAD0000303020103000D000E001000110013000B
:10BAE0001401070108010A010B011C011D020402D7
:10BAF00005020702080219021A021C021D030103B3
:10BB0000020317000201000504000807000B0A00E9
:10BB10001716001D1C010201010504010E0D011183
:10BB200010011413011716011A19020201020B0A5F
:10BB3000020E0D021110021413021716030504035E
:10BB40000807030B0A030E0D0001020307090A0B85
:10BB50000E0F101112141718191A1B1F2021220082
:10BB6000E5A30011A1A400110000000002000000E4
:10BB7000AABA001100000000CDB1001100000000C1
:08BB800002000000A8BA001148
:020000041FFFDC
:10000000000000003D3D0011D8B80011D4B8001127
:100010003461FF1F0000000000000000000000002D
:1000200000000000000000000000000000000000D0
:1000300000000000000000000000000000000000C0
:1000400000000000000000000000000000000000B0
:1000500000000000000000000000000000000000A0
:100060000000000000000000000000000000000090
:100070000000000000000000000000000000000080
:100080000000000000000000000000000000000070
:100090000000000000000000000000000000000060
:1000A0000000000000000000000000000000000050
:1000B0000000000000000000000000000000000040
:1000C0000000000000000000000000000000000030
:1000D0000000000000000000000000000000000020
:1000E0000000000000000000000000000000000010
:1000F0000000000000000000000000000000000000
:1001000000000000000000000000000000000000EF
:1001100000000000000000000000000000000000DF
:1001200000000000000000000000000000000000CF
:1001300000000000000000000000000000000000BF
:1001400000000000000000000000000000000000AF
:10015000000000000000000000000000000000009F
:10016000000000000000000000000000000000008F
:10017000000000000000000000000000000000007F
:10018000000000000000000000000000000000006F
:10019000F932FF1F5931FF1FC16601000000000046
:1001A000000000000000000000000000000000004F
:1001B000000000000000000000000000000000003F
:1001C000000000000000000000000000000000002F
:1001D000000000000000000000000000000000001F
:1001E000000000000000000000000000000000000F
:1001F00000000000000000000000000000000000FF
:1002000000000000000000000000000000000000EE
:1002100000000000000000000000000000000000DE
:1002200000000000000000000000000000000000CE
:1002300000000000000000000000000000000000BE
:1002400000000000000000000000000000000000AE
:10025000000000000000000000000000000000009E
:10026000000000000000000000000000000000008E
:10027000000000000000000000000000000000007E
:10028000000000000000000000000000000000006E
:10029000000000000000000000000000000000005E
:1002A000000000000000000000000000000000004E
:1002B000000000000000000000000000000000003E
:1002C000000000000000000000000000000000002E
:1002D000000000000000000000000000000000001E
:1002E000000000000000000000000000000000000E
:1002F00000000000000000000000000000000000FE
:1003000000000000000000000000000000000000ED
:1003100000000000000000000000000000000000DD
:1003200000000000000000000000000000000000CD
:1003300000000000000000000000000000000000BD
:1003400000000000000000000000000000000000AD
:10035000000000000000000000000000000000009D
:10036000000000000000000000000000000000008D
:1003700019B20011000000000000000000000000A1
:10038000000000000000000000000000000000006D
:10039000000000000000000000000000000000005D
:1003A0000000000000000000000000000D1BFF1F07
:1003B000000000000000000000000000000000003D
:1003C000000000000000000000000000000000002D
:1003D000000000000000000000000000000000001D
:1003E000000000000000000000000000000000000D
:1003F00000000000000000000000000000000000FD
:08183800006FFF1F4118FF1FA4
:10184000024981F3088802F067FB0000006FFF1F68
:1018500070B500241E491F4A1F484C6308CA1B0567
:101860001B0DE4188242F9D11C4B80228B630021AE
:1018700009201B4B920519621A4B1B4DDA671B4B53
:10188000DA688243DA609A68194802409A60112047
:10189000296002F08DF8112002F06AF880226B6C4A
:1018A000112093436B64EE23DB006343114A1B0C4E
:1018B00013840122104B9A7201F004FC0F4B1B7829
:1018C000002B04D10E4B1021187802F0F5F970BDF1
:1018D000000005408805054000060540FF010000A6
:1018E00000F0004004E100E0003800403CF000401F
:1018F000FFDFFFFF0461FF1FB861FF1FE663FF1FEB
:10190000E461FF1F10B502F0F7FA072804D012288F
:1019100008D0022808D010BD044A0420136B0133FC
:101920001363F8E70220F6E71420F4E7DC64FF1FF6
:10193000F8B507000C0026002500503630785135E8
:10194000002804D10300287058342370F8BD29788A
:10195000CA00481E8141A3183800A25C5B68C9B266
:10196000FFF7D0FF00280DD12B78DA00A218013341
:1019700050602B703378044A013B3370136A013393
:101980001362D8E70123DFE7DC64FF1F5C234343D6
:10199000074910B5C9180B0058331B78012B05D126
:1019A000FFF7C6FF034A936A0133936210BDC04636
:1019B0001065FF1FDC64FF1F10B502F06DFA064AC8
:1019C0000121130010CB4942D967044B136002F088
:1019D000DBF9200010BDC04600E100E0100010005F
:1019E00010B5040002F058FA024B1C6002F0CCF96A
:1019F00010BDC04600E100E0431E5A425341A02200
:101A0000F0B5D2015B421340154D164A40019B18B8
:101A10002A18127E8BB00191002A1BD01A000832BE
:101A2000D46F0022E6B206AFE4B294420EDC28186E
:101A3000C369002B08D0019902AA117106AA049269
:101A400002AA167303A898470BB0F0BD1978B954D1
:101A50000132EAE71A7D1A7806AB01261A70E6E72A
:101A60009C67FF1F00400040F0B5254B040040017B
:101A7000C25C85B0002A2BD01A18117E002927D00D
:101A8000917E002924D01179022921D11689D78885
:101A9000D168F51BADB22A1C102D00D9102292B2CC
:101AA000BE4217D11818012303710023C269C380F5
:101AB00003819A4206D068460321037301710293A1
:101AC00001A890470820002C00D0192001F0FAFA54
:101AD00005B0F0BD013C65426C41A0256442ED01BA
:101AE0002C40084D1B186419074D0633013A92B279
:101AF000AA42EDD01888461C1E80085C2070F5E7CD
:101B00009C67FF1F00400040FFFF00000F220E4BAC
:101B100010B59868104002380A280BD801F0FEFF73
:101B20000D0A0B0A0A110A0A0A0A060002210020FD
:101B3000FFF762FF10BD0121F9E70020FFF794FFD6
:101B4000F8E7DB6FF6E7C046004000400F220E4B7F
:101B500010B59868104002380A280BD801F0DEFF53
:101B60000E0A0B0A0A120A0A0A0A060002210120BA
:101B7000FFF742FF10BD01210800F9E70120FFF740
:101B800073FFF7E7DB6FF5E70090004013B5334CC8
:101B90002378072B3DD8324B1A78324B002A39D1A3
:101BA0008022196852020A431A60252001F0C0FE03
:101BB00020232D4A11680B43802113606B460422B9
:101BC000C90508680733104228D080210422C905BE
:101BD000C86810422ED080212020C905CA688243DF
:101BE000CA6014221A701A78002A2FD18021C905E0
:101BF000C86820320243CA6014221A701A78002A78
:101C000028D11A4B1A7D22785A601D221A70593237
:101C1000DA6013BD1A6816490A40C5E7086802432E
:101C20000A6014221A701A78002ACED01A78013A63
:101C3000D2B2F7E7C8680243CA6014221A70197852
:101C40004A1ED2B21A700029F9D1C4E71A78013AB3
:101C5000D2B2C7E71A78013AD2B2CEE73C43FF1FAF
:101C60000444FF1F3CF000403443FF1F00200040AD
:101C7000FFFFFEFF564B70B51B68012B03D1554A81
:101C8000936D0133936502F04FF9534B534A18603B
:101C9000534B544C1A600123534A1360534A136048
:101CA0002378002B06D006225149524802F08CF8C6
:101CB00000232370504A514B10681B78C1B2002B8F
:101CC0000ED14F4CC0B223785BB2002B4FDB237890
:101CD00024785BB264B21B0424021B191B18136026
:101CE0000B1C50294ED95023464A47491078DBB285
:101CF000FF2202284BD10868444C454D267890437A
:101D00002A78964254D9227824782E78023B5D10A6
:101D1000A31B6B435201D31A10335B1118430860A5
:101D200001F0F2FF031F012B45D83A4B1B78002B23
:101D300006D0394B1B78002B02D0002001F00CFF9D
:101D4000A122364B92009978354B4A431B689B1869
:101D5000832292009B181B78033B012B03D8AF20F2
:101D6000400002F021F801222E4BDA8270BD237868
:101D700024785BB264B2FF33FF341B0424021B19C6
:101D80000138ABE7CAB2022AAED20223ACE7086838
:101D9000254C264D267890432A78964208D92278F9
:101DA00024782D78023B5B10641B63435201B2E739
:101DB0002378DBB2B2E70228D5D11D4B1B78013B5B
:101DC000022B03D91B4B1B78022BCCD16C20C8E70C
:101DD0009809FF1FFC0FFF1F2864FF1FFF3F000033
:101DE000141003402C64FF1F0C100340001003402C
:101DF000D50BFF1F7211FF1FB40003408C09FF1F9A
:101E0000680AFF1F490AFF1F94000340460AFF1F8C
:101E1000470AFF1FF908FF1F2209FF1F300DFF1F90
:101E20003409FF1FBC0BFF1F440AFF1F450AFF1F99
:101E30001C09FF1F2309FF1F10B501F0EDFE002252
:101E4000014B1A8010BDC0462464FF1F10B502F07C
:101E50005BF8A121054A89009478054A614312681C
:101E6000044B5218528C1A8010BDC046300DFF1F13
:101E70003409FF1F2464FF1F10B50D4B0D4A9978DC
:101E8000A1239B004B431268D218531DD97F0A4BE4
:101E90001B88994209D2441C07D0C82805D0D269B2
:101EA0005B1A5A43054B5343C01802F0BDF810BDEE
:101EB000300DFF1F3409FF1F2464FF1F7102000053
:101EC00070B5244D2B68002B28D001F095FF2B68AE
:101ED000D8402B680400002B27D002F045F82B686F
:101EE000D8401D4B1D4A9978A1239B004B43126893
:101EF000D118D25C91239B00002A20D0CA5801320D
:101F0000CA50174B17491B680868834214D3D23B49
:101F1000181A012A1AD0144B186070BD01F06CFF1A
:101F2000124B196801F078FFD3E702F01DF80F4B50
:101F3000196801F071FFD4E70D495B18E8E7CA5052
:101F40000C4B1B68DB68E418201AE4E7F530FF301F
:101F5000E1E7C0461C08FF1F300DFF1F3409FF1FBB
:101F60009C09FF1F2864FF1FA009FF1F1808FF1FFF
:101F70002DFF3F003064FF1F70B504000D002829BD
:101F800016D10300A433C2881B889B1A0B4A9BB24C
:101F900093420DD906006A3605223100653001F002
:101FA00023FF002804D13100200001F01DFE70BD88
:101FB0002900200001F0B8FEF9E7C046FE7F0000CE
:101FC000F8B50500012001F057FF134CA36AA26A7F
:101FD0009342FBD1114E336001F0AEFE1049030075
:101FE00008601048426894460F4A17680022BC45B2
:101FF00001D24268BA1A0D4802603268AD18A422B4
:10200000E562606A520302436262094A1278002A5A
:1020100001D00F3B0B60F8BD00F00040340AFF1FF9
:10202000E408FF1F28100040180AFF1F1C0AFF1FAA
:102030001C09FF1F70B580241025E405A3682B43FD
:10204000A36001F091FEA368AB43A36070BD0000E4
:10205000F7B5160080221C001023D205019191686B
:1020600005000B43936000225A4BD7301A6001F0F1
:10207000E3FF9D232A002F009B00EB58CA32012169
:102080000092FC37002B01D00021009A386801F043
:102090001BFE2900009BCB311A784F4BD3351A60B9
:1020A0004B780A781B0213438A7812041A43CB78C0
:1020B0001B061343494A1BBA13604B790A791B026A
:1020C00013438A7912041A43CB7931001B06134358
:1020D000434A1BBA13606B782A781B021343AA7811
:1020E00012041A43EB781B0613433E4A1BBA1360D3
:1020F000019A330213433C4A13603C4B22001B1BE2
:102100009C4603293DDCB3089A0013005142B21AE1
:10211000032A46D1354AE018511A827840781204D1
:1021200000020243E05C043302430A600022FF2BFA
:102130004BDDF0222E4B12011A600F222D4B1A603C
:102140002D4A1368002BFCD00023224A2749136034
:10215000091B321D0B191B68043A180A23706070A2
:10216000180C1B0EA070E3700434002AF2DC8022ED
:1021700010213B68D20501333B6093688B43936029
:10218000F7BD6346D578981893782D061B042B432A
:10219000157804392B43557804322D022B43036004
:1021A000AFE7022A0AD1114AE05C511AE2185278CC
:1021B000120202430A6004339BB2B7E7012AB5D189
:1021C0000A4A521AE15C1160F5E7084959180A6099
:1021D0000433ACE7000004403C00044038000440F5
:1021E00034000440300004400C000440000104406E
:1021F000040004401000044014000440F7B515002A
:1022000080221C001023D2050091916807000B4327
:1022100093600023654AD730136001F00DFF9D23C2
:102220003E009B00F9583B00CA363200FC330029BF
:1022300000D07FE0586801F047FD390032785C4BF0
:10224000CB311A604B780A781B0213438A78AC466C
:1022500012041A43CB78281D1B061343554A1BBA98
:1022600013604B790A791B0213438A7912041A43CB
:10227000CB791B061343504A1BBA13604B7A0A7A78
:102280001B0213438A7A12041A43CB7A21001B06DD
:1022900013434A4A1BBA1360009A2B021343484A5D
:1022A00013602200474B1B1B0093009BCE785B18EA
:1022B00001938B7836061B0433430E78043833437E
:1022C0004E78043136023343019E33600328ECDC40
:1022D0000321A808431C9B002940800003292BD11F
:1022E0003849E5185E18A9786D78E35C09042D0279
:1022F000294319433160030008330021FF2B2DDDF2
:10230000314B324919600F21314B196001232749A4
:102310000B60304B19680029FCD006211B680B406C
:10232000042B20D080220020D20593680A318B43F1
:102330009360FEBD01217DE7022908D121495D1886
:10234000E1184978E35C090219432960D3E70129C0
:10235000D3D11C495918E35C0B60CCE71948181815
:1023600001600433CAE7002310490B606346002B69
:102370000CDC3B00FC335A68102101325A60802289
:10238000D205936801208B439360D2E7009B9B1892
:102390001B68190A13705170190C1B0ED37004239B
:1023A0005B4291709C440432E0E7C0460000044068
:1023B0003C00044038000440340004403000044035
:1023C0000C0004400001044004000440080F000019
:1023D000100004401400044070B5061E19D00222FB
:1023E0005A4B9B799343012B13D1594B1A78FF2AEF
:1023F0000FD15A78FF2A0CD19A78FF2A09D1DA78BE
:10240000FF2A06D11A79FF2A03D15B79FF2B00D16D
:1024100099E0504B0C201A78012A08D000224E4D2A
:102420001A7029780B00093B042B01D8212070BDBC
:102430004B1F012BFAD9454CA37B042B00D982E01A
:10244000A279032A00D97EE09A1ED2B2012A02D8CC
:1024500060881F2877D9002E56D0012E73D1A0880E
:102460000128E3D0002907D1581E032803D801F022
:1024700055FB121715122E702978481E032811D803
:102480000025364B1D602823237501F0FDFCA84272
:1024900027D0A580CAE702212970EDE70421FBE7D8
:1024A0000321F9E707390129C0D82D490968C96A0C
:1024B0008906BBD52B4908780028B7D1012A01D954
:1024C000002BB3D102230B708021274D26338901C5
:1024D0002878237501F000FD80212878890101F01A
:1024E000EBFB0123A380214B1B78002B0AD0FA229F
:1024F00080211F4B92001B8809025A431A4B1878FF
:1025000001F0D2FC002092E701F0C6FC2B78A680F7
:10251000073B012B03D917482E7001F06DFB114BBF
:10252000114C1A78002A06D08021002220788901D7
:102530001A7001F0D1FC01F027FC802120780902FB
:1025400001F0CAFCDEE7122071E7C046A60BFF1FB0
:102550006B09FF1F1A09FF1F1C09FF1F4809FF1FF6
:102560003064FF1F2309FF1F1B09FF1F2109FF1FE5
:102570002C09FF1F0010004010B5002901D001F008
:102580007BFB10BDF7B5604B01919978A1239B00AF
:102590004B435E4A060014681022E418D6235B0001
:1025A000E0583623FF33E35C00279343222B41D1CD
:1025B000574B0F3A1A600760012501F00DFC019B93
:1025C0001880E8235B00E35C002B01D0B34258DDA8
:1025D0000023504FFB70AD33FF33E3581A68002AD5
:1025E00003D09B88DB439B071DD03823FF33E35C7C
:1025F000002B18D09B235B00E35C002B13D1D1335D
:10260000FF33E35CB3420EDAA4235B00E15AE01827
:10261000090A023101F000FD23000122FE33013ED0
:1026200001351A87FA70E8235B00E35C002B2AD09F
:10263000A8B2FEBD03683D00002BBED081880430E7
:10264000090A023101F0E8FCD6235B00E3581F6061
:10265000B2E72300B133BA00FF33985801378188BD
:102660000430090A023101F0D7FCE8235B00E35C87
:10267000BB42EEDCE822F61AED1800235200A35408
:10268000A6E70027F1E7200001F0DEFB00281FD0BD
:10269000002E1DDD7319882647190193B60020000E
:1026A00001F072FA5A3080002018406801358188A4
:1026B0000430090A023101F0AFFC200001F044FCB3
:1026C000A3590133A351BD4202D0019B9D42E6D1E3
:1026D000114BE35C002BABD095239B00E35C002BFC
:1026E000A6D00E4BE15A0029A2D00D4AA35C994214
:1026F00002D90133A3549BE700231A212000A354DD
:1027000001F04AFA94E7C046300DFF1F3409FF1F5D
:1027100000140340E010FF1F5A0200007202000084
:102720005E0200000D4970B54A6E0D4CD2038B69F4
:10273000D20BA24206D80B4D0224AA4204D901F0C2
:1027400003FB70BD02246442E21815007E2425407C
:102750002242F4D0A3432B438B61F0E700F000400A
:102760000A200000FC1C0000F8B51D4B1D4F1A7814
:10277000002A10D1BA7B002A02D101321A7003E07C
:10278000032AFAD0022AF8D001F07EFB00220120B1
:10279000154B1A70F8BD154B154D1C68154B9E78DE
:1027A00001232B702878C0B200F09EFBBB7B002B6E
:1027B0000BD101F089FBA1239B007343E418832311
:1027C0009B00E41823782B70E4E7032B02D101F07F
:1027D00063FAF0E70020022BDCD101F0E5FBEAE729
:1027E0001C09FF1FA60BFF1F2309FF1F3409FF1F32
:1027F000490AFF1F300DFF1FF0B587B00EAD2F78CF
:102800000FAD2D780593AC46634614000E4D0CAA0F
:1028100012782E7803930D9B009201932200059B62
:10282000029701F001FB2E70012C01D0042C08D17D
:10283000802206498B889343054A1278D2011343BC
:102840008B8007B0F0BDC0461C09FF1F6C11FF1F35
:102850007809FF1F0B001B3B70B504003020E02BF4
:102860000DD81300E025493BFF3B9BB2ED00AB4286
:1028700005D8034B200019825A8201F095F970BDEA
:102880008410FF1F10B501F04FFB054B00205B6863
:10289000052B04D9034A5268D20200D4980810BD0F
:1028A00000100040FCE100E070B501F0F5FA0D4BBE
:1028B0001B68FC33DC691D6AFFF7E4FF641984427E
:1028C00004D2094B01241B68002B07D004220024EA
:1028D000064B1A70064A93690133936101F054FA6A
:1028E000200070BD3064FF1F9809FF1F2309FF1FE0
:1028F000FC0FFF1F70B50C4D2B68FC335C6A01F0B8
:10290000CBFAFFF7BFFF2B680025FC339B6AE31867
:10291000834204D2054B1B68AB4200D1051B01F07A
:1029200033FA280070BDC0463064FF1F9809FF1FAE
:10293000D722044B92009B5810B5002B00D098472B
:1029400010BDC0460000FF1F10B501F0CFF8FFF723
:10295000EFFF2749274BCA6D274C1A4084235B00A1
:102960001343CB65254B1B68186A01F085FA244B8D
:10297000244A1A60244B254A1A60A022244B520094
:102980001A60244B187801F0A7F92000224901F0C1
:10299000ABF90023A3600233A360204B20492360DE
:1029A00003232048A36001F09FF910221E4BFF2053
:1029B0001A60802252031A60802292031A608022D9
:1029C00012041A6001F0C8F8012001F0CDF8FA20D5
:1029D000400001F091F9582001F0E6F9134801F0A8
:1029E000CBF9012001F040FA072001F0B5F910BD44
:1029F00000F0004000FEFEFF141000403064FF1F96
:102A0000000003400180063DBC0003403408000084
:102A1000A40003404A0AFF1F71020000C30900001E
:102A2000FFFF3F002810004000E100E0307500008B
:102A3000674E336888331B6883F3088801F0CCF84D
:102A4000644A6549136800200B401360634B644A75
:102A50001B68934200D1A6E001F0E6F80221614A2A
:102A600013688B431360FFF76FFF5F4B5F4C187861
:102A7000C0B201F0C9FA0023A3600233A3605C4B2B
:102A80000120236001F0F8F90323A36001F0BCF8F2
:102A9000040001F049FA050001F0B6F8554B186042
:102AA00001F08AF8544B1968621A531EA14200D2F1
:102AB00013008022D203934201D39B029B0A326807
:102AC000D16AC90700D471E04C491C0C09689BB25B
:102AD0004C4359432402090A641803264849FC322E
:102AE00093680A6847489B1A474A0768126847492B
:102AF0009B18474A9A1833409208DB190A60036012
:102B0000042B03D9013233400A6003600E68414947
:102B1000A619300001F080F93F4F3E493B68C318C9
:102B20003B603000019301F097F93C4E3068081883
:102B300038493060884205D9019B01333B6001F080
:102B40008BF9316001F078F8354B1B78002B0DD0F4
:102B500001F0EAF9334B621B196812188A4232D22B
:102B60004919091B091A304801F0BEF82F4E337A73
:102B7000002B0ED001F0D8F9621BF16812189142B7
:102B800024D94919091B091A294801F0ADF8002375
:102B90003372284B83F3088801F0DEF9002001F03E
:102BA00043F801F0E9F901F03FF85CE7DC01990036
:102BB0000234641A5900641A09214B438033CB4014
:102BC000A408E41889E7FA218900CCE71A49DBE771
:102BD0003064FF1F1CF00040FFFFC1FF0C0AFF1F05
:102BE000B641210310000040490AFF1F14100040A5
:102BF000C3090000100AFF1F340AFF1F380AFF1F15
:102C0000200AFF1F280AFF1F1C0AFF1F240AFF1F9C
:102C1000C4090000710200006008FF1F2C0AFF1F9A
:102C20001C09FF1FE408FF1F00100040740BFF1F6A
:102C30003C10004000000020DC050000A022054BF5
:102C400092009B5810B5002B01D0984710BD01F0A1
:102C5000DBF8FBE70000FF1FA122054B92009B5809
:102C600010B5002B01D0984710BD01F0CDF8FBE75F
:102C70000000FF1FA222054B92009B5810B5002BAD
:102C800001D0984710BD01F0BFF8FBE70000FF1F1F
:102C9000A322054B92009B5810B5002B01D09847FA
:102CA00010BD01F0B1F8FBE70000FF1FA422054BA7
:102CB00092009B5810B5002B01D0984710BD01F031
:102CC000A3F8FBE70000FF1F70B501F02DF94F4B93
:102CD000186001F089F90400C30702D401F054F927
:102CE00070BD00224A4B1A604A4B187801380428FC
:102CF00029D800F013FF0320181C2400200000F046
:102D0000B3FF0128ECD0444C2378042B6ED101F0A2
:102D1000EBF80028E4D000F0C7FF582001F044F899
:102D200002232370DCE7200001F04EF9E9E72000E0
:102D300001F052F9E5E7200001F05EF9E1E720003B
:102D400001F02AF9DDE700F0DFFF0500012808D1D6
:102D5000324B1B78053B012B03D82000FFF76EFF99
:102D6000D1E72D4B1B78022B01D0052B20D1022D52
:102D700028D12B4B9B7BAB431CD12000FFF76CFF72
:102D8000264B18780128BED16405BCD424492522DD
:102D90004B7B034205D1233A13405A425341263319
:102DA0001A000B7D9342AED9322001F005F9AAE753
:102DB000022D07D1194B1B78052B11D12000FFF7ED
:102DC00059FFDDE7012D0BD1012B03D12000FFF7C7
:102DD0005FFF98E7062B03D12000FFF767FF92E71C
:102DE000200001F011F8022D8DD1C9E7032B04D189
:102DF0000C4B987C00F030FF72E7072B00D06FE798
:102E0000094B987B00F0C8FF6AE7C0469C09FF1F8A
:102E10009809FF1F9009FF1F2309FF1F1C09FF1FAF
:102E2000A60BFF1FBC0BFF1FD40BFF1FFA210A4B81
:102E30000A4A49001A640A4A5A500A4A04395A503E
:102E4000094A08319A64094A5A50094A5C315A5071
:102E5000084ADA667047C0460000FF1FF927FF1FC7
:102E6000F528FF1FA928FF1FD923FF1F6927FF1F70
:102E7000791EFF1F4D1EFF1FF7B50B0CFF27012208
:102E8000009300233C001E001D009446019089B26F
:102E900062469A401000084018413618B6B2FF2F1B
:102EA00002D1012E00D19FB2009802401A41AD1804
:102EB000ADB2FF2C02D1012D00D19CB20133102BF9
:102EC000E6D10320012E07D1012D04D1019B24015D
:102ED000E4191C700138FEBD102EFCD10238102DF3
:102EE000F9D00230F7E700008023F7B59C46264B67
:102EF000264F01932649274A274D284C284B022864
:102F00001AD1604638600868264E30408026360365
:102F10003043086001990978002909D11660224AD6
:102F20002A60224A2260E02219689143A03A1BE0FD
:102F30008021C9021160F2E766463E600F68194EB3
:102F40003E408027FF023E430E6001990978002928
:102F50000DD1176001280ED1154A2A60154A22604A
:102F6000E02219689143C03A0A431A60F7BD8021F4
:102F700089021160EEE7E0210F4A02432A600F4AFE
:102F800022601A688A43F0E74B0AFF1FE000034003
:102F9000D80003409000034000000340500003406D
:102FA00040000340FFFFE3FF0280063D804508220A
:102FB0000180063D80660822008006988055082220
:102FC000F8B51E4B80261A680020140034403242A7
:102FD00032D11A681A4F32431A6001223B68063018
:102FE00093433B6000F048FF0122164D2B681E43BF
:102FF0002E603B680A2613433B608027BF00124BBC
:103000001B683B4211D1013EF6B2FF2E09D17E2250
:103010000E4B1C682B68E40B1440934323432B6036
:1030200005E0082000F028FFE9E7002EEFD180221C
:103030002B68600893432B60F8BDC046C4F0004085
:103040005CF0004018F0004068F0004060F0004084
:1030500010B500F091FD01215820034A00F0ECFE6C
:10306000FFF7AEFF10BDC046600AFF1F10B5782203
:103070000021034800F0A0FE00F0E6FD002010BD96
:103080002467FF1F70B5040000F006FF00230C202A
:103090000B4A010059438D18515C00290DD0A14203
:1030A00008D1012300246B7000F006FF00F06CFED5
:1030B000200070BD01330A2BEBD11224F6E7C04685
:1030C0002467FF1F70B5040000F0E6FE002319001E
:1030D0001D000D4A1078002806D0A0420CD1557072
:1030E00001310C320A29F5D1002B0AD100F0ACFDD8
:1030F00000F04AFE002070BD5078461EB0411B18FB
:10310000EEE700F0D9FEF3E72467FF1FF7B50400F0
:103110000C20002384460E4D019267465F43E85D14
:103120007E19A04212D000280BD10A4B9C46624661
:103130001B7808331370019B70707C557160B3600D
:10314000FEBD01330A2BE8D10320F9E70720F7E79A
:103150002467FF1F2067FF1F8020F8B5484BC0057C
:103160001B68C1248360474BFF251A680123134362
:103170004361454BA4001A68444B40211A60444BFC
:103180001A68444B1A60444B1A59AA431A51C52273
:1031900092009E58AE433143802699509F583F4934
:1031A000F6010F403E439E509E5880273602360A55
:1031B0003043985080201A5900020A4002431A51A5
:1031C00004341A59364E3F04324080263A431A518D
:1031D0001A5936061202120A32431A5108341A5981
:1031E00080260A4002431A51C32292009F58B446D7
:1031F000AF4337439F509F58294E0F4007439F507E
:103200009F58374080263604374380269F509F586A
:1032100036063F023F0A37439F50C0221F59AF4333
:103220003A431A511A591202120A1643C6221E5163
:1032300092009C58AC4365462C439C509C580025FA
:103240000C4020439850C72080001A58154C11405C
:10325000C02212020A431A50134B1B78DB08AB4200
:1032600001DC0020F8BD2378002B06D0A368002BDA
:1032700000D0984701350C34EEE71220F2E7C04643
:103280003843FF1F3443FF1FB0F000401C67FF1F8F
:10329000B4F000401867FF1F00E100E0FF00FFFFEF
:1032A000FFFF00FF2467FF1F2067FF1F030010B50B
:1032B0001F2809D8072200201340072404490A7850
:1032C000A24313430B7010BD00230620F5E7C04650
:1032D0002067FF1F054B06491B780A6805485B07F6
:1032E00002401B0B134300200B6070472067FF1F39
:1032F0001CF00040FFFFC1FF70B50C25FFF7EAFF8F
:103300000A4B1C780A4BE4086543ED18002C01D1E8
:10331000200070BD2B78002B06D06B68002B00D0EE
:103320009847013C0C3DF1E71220F2E72067FF1FB0
:103330001867FF1F1FB5002102220B0001910091A9
:10334000052000F0F9FD02230B490A681A42FCD15E
:1033500020230393039B5A1E0392002BFAD1074AA2
:103360001368002BFCDA0B246C442000012100F0D0
:10337000EBFB207804B010BD90C8004000C80040AE
:1033800013B504000A4B0193019B002B01D11120BE
:1033900016BDFFF7CFFF23000340044205D00520F0
:1033A00000F06AFD019B013BEDE71800F0E7C04625
:1033B000FFFFFF0707B500F06FFD80220821D2054F
:1033C000936A0191002B01D10739916202210C4AC5
:1033D00011600199481E01900029FAD10331116052
:1033E000053101910199481E01900029FAD111601F
:1033F000002B02D18022D205936200F0C5FC07BDEC
:1034000000C00040F0B52D4C89B02378002B4FD17F
:10341000FEF7D2FA02232A4F03903A681A42FCD1EF
:1034200020230693069B5A1E0692002BFAD1254EA6
:103430003368002BFCDA0120FFF7A2FF011E02D047
:10344000112009B0F0BD030003220190009005ADEA
:103450009F2000F071FD0321280000F075FB02237E
:103460003A681A42FCD120230793079B5A1E079201
:10347000002BFAD13368002BFCDA0120FFF780FF24
:103480000028DDD10398FEF7ABFAAA786B78110417
:103490001B020B4329780B4363601300113B0A495D
:1034A000052B07D801239340A3600B6001232370F1
:1034B0000020C6E780231B03F6E7C0462043FF1F1A
:1034C00090C8004000C800409808FF1F1E4B30B550
:1034D0005A6818781D4B85B0D31859424B410121C9
:1034E0000093002300F0D0FB194B1A4A02259A637F
:1034F00000221A6510325A658022C4219D65164B40
:103500001648D202DA6789004258154B80241A40C7
:1035100080231B0413434350642341200393E40599
:1035200000F006FA402000F003FA6562039D6B1E6E
:103530000393002DFAD103236362FFF73BFFA562DB
:10354000FFF760FF05B030BD2C43FF1F95FFFEF76E
:1035500000C80040050001FF04E100E000E100E0D8
:10356000FFFF00FFF0B585B00700FEF725FA022344
:1035700005002D4C22681A42FCD120230093009BA9
:103580005A1E0092002BFAD1284E3368002BFCDA29
:103590000120FFF7F5FE002803D01124200005B01C
:1035A000F0BD234B2360022322681A42FCD1202362
:1035B0000193019B5A1E0192002BFAD13368002B14
:1035C000FCDA0120FFF7DCFE0028E6D1194B1F6072
:1035D000022322681A42FCD120230293029B5A1E26
:1035E0000292002BFAD13368002BFCDA0120FFF79E
:1035F000C7FE0028D1D1104B2360022322681A4253
:10360000FCD120230393039B5A1E0392002BFAD173
:103610003368002BFCDA0120FFF7B2FE041EBCD198
:103620002800FEF7DDF9B9E790C8004000C8004067
:1036300001000006A8C800400180000110B500206C
:10364000FFF790FF10BD000010B5064B18705960D1
:10365000FFF73CFF00211320034AFFF757FD00202E
:1036600010BDC0462C43FF1FCD34FF1FF0B5040032
:1036700085B003920291FEF79FF9882263035B0BEA
:1036800052051A438023DB059D6A8023274F009251
:10369000BA68002601901B039A420CD9F823260031
:1036A0001B041E401C4206D08022214B52025E6247
:1036B00019680A431A60002D0BD100F0EDFB0222BD
:1036C0001C4B1A608023DB055A62013A9A6200F0B3
:1036D0005BFB0023039A934220D1002D0AD100F016
:1036E000DBFB144B03221D608023DB055A629D62C5
:1036F00000F04AFB8023BA681B039A4208D9002EC7
:1037000006D000220A4B0C495A621A680A401A6015
:103710000198FEF765F9002005B0F0BD009A029906
:10372000D2181278CA540133D4E7C0462043FF1F91
:1037300000C8004000C00040FFFFFEFFF0B587B0AA
:10374000029103920400FEF737F9019000F0A4FB08
:10375000802302250122234EDB0535605D629A62DB
:1037600000F012FB204F3B682B42FCD12023049336
:10377000049B5A1E0492002BFAD11C4D2B68002B7F
:10378000FCDA0120FFF7FCFD002802D0112007B071
:10379000F0BD2000039A029900F0BEFA0223040053
:1037A0003A681A42FCD120230593059B5A1E0592C4
:1037B000002BFAD12B68002BFCDA0120FFF7E0FD8B
:1037C000051EE3D100F068FB80230322DB05356092
:1037D0005A629D6200F0D8FA0198FEF701F9E0B252
:1037E000D5E7C04600C0004090C8004000C8004077
:1037F000F0B5802489B00600FEF7DEF8E405A36A80
:1038000002250393029000F047FB0123304F3D60F7
:103810006562A36200F0B8FA2E4C23682B42FCD1FB
:1038200020230593059B5A1E0592002BFAD12A4DA1
:103830002B68002BFCDA0120FFF7A2FD002803D043
:103840001124200009B0F0BD244B2360022322681C
:103850001A42FCD120230693069B5A1E0692002B87
:10386000FAD12B68002BFCDA0120FFF789FD021E3C
:10387000E6D11B4B03211E60030001900090202025
:1038800000F05AFB022322681A42FCD1202307933E
:10389000079B5A1E0792002BFAD12B68002BFCDAEB
:1038A0000320FFF76DFD041ECAD100F0F5FA802356
:1038B0000322DB053C605A629C6200F065FA039BC0
:1038C000002B01D1FFF776FD0298FEF789F8B8E7E3
:1038D00000C0004090C8004000C800400100000641
:1038E00094C8004007B5000201910422000A01A912
:1038F000FFF724FF0EBD000073B5050005240B4A39
:10390000A3005B429B1819686B46DE1D3000FFF771
:10391000B3FA022804D133782B55013CEFD276BD9F
:10392000052CFCD00128FAD10230F8E71409001167
:103930001F2807D8012380228340D20591680B43BA
:10394000936070473F2808D80123802220388340A5
:10395000D20551690B435361F3E75F28F1D8012386
:10396000802240388340D205116A0B431362E8E796
:103970001F2807D8012280218240C9058B68934304
:103980008B6070473F2808D8012280212038824070
:10399000C9054B6993434B61F3E75F28F1D80122D6
:1039A000802140388240C9050B6A93430B62E8E7E7
:1039B0001F2810D880230200DB05153A1968012A58
:1039C00006D820229143196019680A431A6070478B
:1039D00001228240F6E73F2811D880230200DB0550
:1039E000353AD968032A06D810229143D960D9689C
:1039F0000A43DA60EBE7012220388240F5E75F28CE
:103A0000E5D842238022181A413B8340D205516AEF
:103A100099435162516A0B435362D8E710B50400D1
:103A2000012813D1A022184992050B685B015B099C
:103A300013430B60154B164A19681140154A0A4387
:103A40001A60402219680A431A6010BD0028FCD190
:103A500001000A2000F0B8F821000B2000F0B4F8B3
:103A6000C0220A4B920019680A4340211A601A6862
:103A70008A431A60B022044912060B685B015B0995
:103A800013430B60E1E7C04614F000401CF0004017
:103A90007F00FEFF80FD010072B6074A1368013304
:103AA00013600422054B1A600023054A136080222C
:103AB000D2055360FEE7C0467808FF1FC0F0004003
:103AC000C4F0004005490B68002B05D1044A0A6088
:103AD00004490A60044A13607047C046140AFF1F75
:103AE000841E0000380AFF1FC4F000400023034A70
:103AF0001360034A1360034A1360704754F0004098
:103B000040F1004044F1004002B4714649084900C8
:103B1000095649008E4402BC7047C04602B4714643
:103B200049084900095C49008E4402BC7047C04600
:103B300003B47146490840004900095A49008E44BF
:103B400003BC70470000000001B40248844601BC79
:103B5000604700BF3D71010001B40248844601BCCA
:103B6000604700BFED6B010001B40248844601BC10
:103B7000604700BF6911010001B40248844601BCDE
:103B8000604700BFED68010001B40248844601BCF3
:103B9000604700BFD9B0000001B40248844601BCB0
:103BA000604700BF53B9000001B40248844601BC1D
:103BB000604700BF116E000001B40248844601BC9A
:103BC000604700BFC166010001B40248844601BCE1
:103BD000604700BF799E001101B40248844601BCD1
:103BE000604700BFC9A9000001B40248844601BC77
:103BF000604700BF85C1000001B40248844601BC93
:103C0000604700BFC1A5000001B40248844601BC62
:103C1000604700BF156B010001B40248844601BC37
:103C2000604700BF8D82000001B40248844601BC99
:103C3000604700BF016C010001B40248844601BC2A
:103C4000604700BFD544010001B40248844601BC6E
:103C5000604700BFADAE000001B40248844601BC1D
:103C6000604700BF4DF9000001B40248844601BC22
:103C7000604700BF0134010001B40248844601BC22
:103C8000604700BFE9D4000001B40248844601BC8B
:103C9000604700BFC56D010001B40248844601BC05
:103CA000604700BF75F8000001B40248844601BCBB
:103CB000604700BF6DF6000001B40248844601BCB5
:103CC000604700BF0D52010001B40248844601BCA8
:103CD000604700BF2144000001B40248844601BC93
:103CE000604700BFEDA5000001B40248844601BC56
:103CF000604700BF2D6C010001B40248844601BC3E
:103D0000604700BF8512010001B40248844601BC2F
:103D1000604700BFDD0C010001B40248844601BCCD
:103D2000604700BF9573010001B40248844601BC9E
:103D3000604700BF51B8000001B40248844601BC8E
:103D4000604700BFBD5C010001B40248844601BC6D
:103D5000604700BFD1AE000001B40248844601BCF8
:103D6000604700BFF90D010001B40248844601BC60
:103D7000604700BFDD3F000001B40248844601BC3B
:103D8000604700BF8D11010001B40248844601BCA8
:103D9000604700BF9DA9000001B40248844601BCF1
:103DA000604700BFC1F7000001B40248844601BC6F
:103DB000604700BF7912010001B40248844601BC8B
:103DC000604700BFB70E000001B40248844601BC42
:103DD000604700BFE94C010001B40248844601BCC1
:103DE000604700BFCD0C010001B40248844601BC0D
:103DF000604700BFCD4C010001B40248844601BCBD
:103E0000604700BFE90B010001B40248844601BCD1
:103E1000604700BFE917010001B40248844601BCB5
:103E2000604700BF090E000001B40248844601BC8F
:103E3000604700BF9D6A000001B40248844601BC8F
:103E4000604700BF0167010001B40248844601BC1D
:103E5000604700BF71B0000001B40248844601BC55
:103E6000604700BF090E000001B40248844601BC4F
:103E7000604700BFE512010001B40248844601BC5E
:103E8000604700BF0189000001B40248844601BCBC
:103E9000604700BFA9D8000001B40248844601BCB5
:103EA000604700BF75A9000001B40248844601BC08
:103EB000604700BF8B52010001B40248844601BC38
:103EC000604700BF21A9000001B40248844601BC3C
:103ED000604700BFE9F6000001B40248844601BC17
:103EE000604700BFB352010001B40248844601BCE0
:103EF000604700BF01D7000001B40248844601BCFE
:103F0000604700BFE927000001B40248844601BCB5
:103F1000604700BFF9ED000001B40248844601BCCF
:103F2000604700BF21B2001101B40248844601BCC1
:103F3000604700BFC95C010001B40248844601BC6F
:103F4000604700BF496D010001B40248844601BCCE
:103F5000604700BF5976010001B40248844601BCA5
:103F6000604700BF7997000001B40248844601BC55
:103F7000604700BF6D0B010001B40248844601BCDC
:103F8000604700BF8552010001B40248844601BC6D
:103F9000604700BFDD0A010001B40248844601BC4D
:103FA000604700BFF935010001B40248844601BCF6
:103FB000604700BF19FA000001B40248844601BC02
:103FC000604700BF6137010001B40248844601BC6C
:103FD000604700BF0934010001B40248844601BCB7
:103FE000604700BF0534010001B40248844601BCAB
:103FF000604700BFBD0B010001B40248844601BC0C
:10400000604700BFF535010001B40248844601BC99
:10401000604700BF8914010001B40248844601BC16
:10402000604700BFC115010001B40248844601BCCD
:10403000604700BF8937010001B40248844601BCD3
:08404000604700BF8944000045
:1040480002000000A6BA001101000000C8B8001163
:1040580002000000A2BA0011010000008840FF1F02
:1040680002000000D0B8001101000000B461FF1F79
:1040780002000000A0BA0011030000002861FF1F21
:104088001200000002000000A6BA001101000000A2
:1040980010B9001102000000A2BA001101000000CE
:1040A8000DB90011020000001AB900110300000048
:1040B8006361FF1F02000000A0BA001103000000A6
:1040C8007861FF1F02000000A2BA00110100000081
:1040D8000CB900110200000018B90011030000001B
:1040E8003961FF1F02000000A0BA001103000000A0
:1040F8005A61FF1F02000000A6BA0011010000006B
:1041080054B9001102000000A2BA00110100000019
:10411800D141FF1F0200000066B900110100000034
:104128004BB9001102000000A2BA00110100000002
:10413800D041FF1F0200000064B900110100000017
:104148008061FF1F02000000A2BA001101000000F8
:10415800CF41FF1F0200000062B9001101000000FA
:104168003BB9001102000000A2BA001101000000D2
:10417800CE41FF1F0200000060B9001101000000DD
:1041880036B9001102000000A2BA001101000000B7
:10419800CD41FF1F020000005EB9001101000000C0
:1041A80031B9001102000000A2BA0011010000009C
:1041B800CC41FF1F020000005CB9001101000000A3
:1041C8002CB90011020202020202000000000000E5
:1041D80016150000154B0011D94A0011B4B9001189
:1041E80090011D0018001800FFFF070102030405D5
:1041F80006020106000000000000000000000000A8
:1042080000000000000000000000000000000000A6
:104218000300000002000000A6BA0011010000001F
:10422800D4B9001102000000A2BA00110100000078
:104238008C42FF1F02000000DEB9001101000000DF
:10424800AE61FF1F02000000A0BA001103000000C9
:104258001864FF1F02000000A2BA0011010000004C
:104268008C42FF1F02000000DCB9001101000000B1
:10427800B061FF1F02000000A0BA00110300000097
:104288001064FF1F1200000000010000000001116F
:10429800FFFF0000504859360000000000000000F1
:1042A8000B000500F0000000B400002800280028DA
:1042B8003075A000A000A000A00000080008E001E0
:1042C800F000100010001000100010001000500046
:1042D8005000500010001000D0070000000000003F
:1042E8000F0001000500307507001000010081FF74
:1042F80000000000FF00000061700011696E0011ED
:10430800F96B0011FFFF0100FF0000007D9A00110A
:10431800F99700111197001100000000000000003B
:1043280000000800040000003B0001085902E001F9
:1043380088212800FF00000002000000A6BA001132
:10434800010000006CBB001102000000A2BA0011BD
:1043580001000000BD43FF1F020000009EBA0011CB
:1043680001000000DC67FF1F02000000A2BA001174
:1043780001000000BC43FF1F020000009CBA0011AE
:1043880001000000BA43FF1F02000000A2BA00119A
:1043980001000000B843FF1F020000009ABA001194
:1043A80001000000B043FF1F180018001D00900115
:1043B800020000030202000002000000A6BA001179
:1043C8000100000080BB001102000000A2BA001129
:1043D800010000000044FF1F0200000098BA00110D
:1043E800000000000000000002000000A0BA001158
:0A43F80003000000FC67FF1F20FF18
:040000051FFF184180
:00000001FF
